:020000041100E9
:103000007FB50023284C294D03932800217C284AB2
:1030100001F0DFFA002812D103232800217C03AA43
:1030200001F07EFA00280AD1224B039A9A4206D177
:10303000214B2248E360224B636104B070BD02263D
:10304000217CFE2228001F4B009601F03BFA00284D
:1030500001D00020F1E71C4BA2899A42F9D1217CD2
:10306000FF222800194B009601F02CFA0028F0D11D
:10307000E389174A934203D1164B17486361DCE793
:10308000164A9342E5D1164B164A1B68934206D95D
:10309000C02304222800217C9B0001F07CFA124B03
:1030A00012486361C9E7C0460C62FF1F3C42FF1F24
:1030B0008137000059595300595983200CBF001122
:1030C000054200111862FF1F595900001A62FF1FC4
:1030D00083050000B9410011ECBE0011821500000B
:1030E0003062FF1F87130000C1420011FCBE0011B7
:1030F000002370B51A4E1B4C30006361637401F0FD
:103100008FF9402323744B2B0CD9CC233821AC22CC
:1031100030009B01217401F03EFA00280AD00025FE
:1031200025740CE0FFF76CFF051E08D1237C0433E7
:10313000DBB2E7E70C4B0D4D63610D4BE381236878
:10314000002B08D1002D06D00C222900200008F009
:103150004FFE2B7B6374300001F0A0F970BDC046B8
:103160003C42FF1F0C62FF1F59420011DCBE0011E0
:10317000AAAAFFFFF7B5164B0192C318021D002043
:10318000009388235B05D3181B685C1C1AD09CB283
:10319000402C18D88D781E0CAC466746CD782D0291
:1031A0003D43AE4206D1019800280ED110000C70AC
:1031B000240A4C7003249BB20733A343D218009B0C
:1031C0009A42DED3FEBD4432F9E71000FAE7C0466A
:1031D000FC0F0000802213B503000324019189B283
:1031E000520107319B18A14304305A1A88235B050A
:1031F000C3181B68591C03D190429241104016BD60
:1032000099B2402907D80B000733A343C018904256
:10321000ECD30020F3E74430F9E7134B134A1B6863
:10322000126810B5FA24934201D81A00F824104B02
:10323000E4021B689A4210D813000E4A12689A42A0
:103240000ED3013307D1F823DB029C4203D10A4994
:10325000054808F0A5FD200010BDFC24E402ECE7C1
:10326000FE24E402F7E7C04600C0071100D00711B2
:1032700000E0071100F00711FFFFFF7FF0B59BB0E2
:10328000150004900391402A00D9A0E006AB5980B4
:103290001A80FFF7C2FF0400042816D9002206A9ED
:1032A000FFF768FF052810D906AB1B88AB420CD18D
:1032B000002D07D0514B2A000499C01808F0A8FA35
:1032C000002802D101201BB0F0BD06AB1D802000FC
:1032D0000699FFF77FFF041E7BD1069B0793FFF73C
:1032E0009CFF80235B01C618802307001B039E42BE
:1032F00001D3F826F60288235B05F31801931B68B7
:10330000013302D0019808F00BFB3D49019808F009
:1033100047FD3B1D0293331D05938822029B5205F6
:103320009B181B6808935A1C3CD044219AB2009108
:10333000402A04D80320D11D814389B2009103990A
:103340001B0C8B4224D0402A22D80122300008A92D
:10335000FFF710FF021E1BD1380008A9FFF70AFF74
:103360000400042831D9009A059B9B188022520141
:10337000B218934240D288235B05C118009A09A86D
:1033800008F036FD1D4B009A09A9F01808F050FB13
:10339000009A029B9446634402931A4B029AFB18CC
:1033A0009A42BAD388235B05FC1821680198013939
:1033B00008F0F6FC200008F0B3FA039A07AB5A8035
:1033C00030000799FFF706FF0400002C03D100200E
:1033D00079E70428FBD988235B05E018069908F0F3
:1033E000DFFC0323EA1C9A4300D16BE7034B0499EB
:1033F000E01808F01DFB65E70424ECE70400001169
:10340000FFFFFF7FF80F0000F7B505001400402A0A
:1034100021D8002701AE71803780FFF7FEFE042817
:1034200016D93A003100FFF7A5FE042810D93688D6
:10343000BC420BD0BD4209D0221CB44200D9321C80
:10344000064B92B2C118280008F0D2FC30B2FEBD83
:10345000C04300B2FBE703204042F8E7040000113C
:1034600037B5042204000D0001A81649FFF7CCFF70
:10347000020004280BD1019BA34208D3AB4204D025
:10348000104901A80195FFF7F9FE01203EBD0E4C41
:1034900023682000019308F043FA019920000139C4
:1034A000019108F07DFC80235B01E418074B9C42EE
:1034B000EED10422034901A80195FFF7DFFE0020A9
:1034C000E4E7C0465555000000C007110000081190
:1034D00030B589B008F0E4FB10226946254808F0B1
:1034E000CFFA254B009A9A420ED1019B029A0F2BDC
:1034F00033D8002101240698013B08D2002900D0CE
:103500000292029B013331D10023029325E0551C26
:10351000F2D102002100EFE710341022200004A9AC
:1035200008F0AEFA029B013301D1069B0293882377
:1035300004995B05C918059B06981A03120B0491A0
:103540000592814203D02B4201D108F051FC019B2E
:10355000013B0193019B002BDED1029B002B03D08A
:10356000049304984168084709B030BDE025014C38
:103570002D03EFE700000111504859368022F8B5BD
:10358000964C974BD200002120001C6008F0B8F93F
:103590002300944A88331A60934B1A786A23002ACE
:1035A00000D01133E3620A232365904B37221B7846
:1035B0000820A3638E4B2118E361102323628D4BF7
:1035C0003B256361C823DB00A36123008C331A60B1
:1035D0002823013AE26320646364CA67043A211D28
:1035E000CA672100BC310D602100C0310860210094
:1035F000C4310B6021000635CC310D602100083D3F
:10360000C8310D602100D0310A602200D432106030
:103610002200D832136022000227E0322100176016
:103620004222DC310A6021001B3DE4310D602100A3
:10363000E83108602100EC310B6023000521F433F0
:1036400019602300F0331A602300183290331A6097
:1036500023009433186023001E3A98331A60AF2376
:10366000DB002360644BFA262363644B644DE36004
:10367000644BF031A3642300FF31FC33B600A1603A
:1036800021611E60A5627325E5656D3D6565A565D3
:1036900096255D4AAD00E264666258606766A5667D
:1036A00000270925A767E566584F594D6067200038
:1036B0002567E2673A6015279C30676007001A208B
:1036C00038602000A0300700212038602000A8309A
:1036D00007004C4838602000F83006602600642758
:1036E000A436376026005F3FAC3637602600033FC4
:1036F000B03637602600C637B4363760260000275C
:10370000B836376038269E60424E96205E64424E40
:103710005A66DE61414E9A645E62F53EFF3E9E62ED
:103720001E269A67354A8000DE661F675F67DD6583
:103730001D661862DA67BE23394A5B00E250394BD6
:10374000D838235004302250C4225200A350C6233C
:10375000E4205B00E1500433334AE1503349344BF9
:10376000D1603449800019503349E938FF38195085
:1037700032490430195032493248D161324911631B
:10378000324951631900F4310860CE2030494000BD
:1037900011603049195019002F48F83108602F493D
:1037A000D16582212E4A89005A501A002D490832CB
:1037B000D1671A002C49B432116088212B4A890044
:1037C0005A501A002A49883211602A4ADA6408F0ED
:1037D00017F8012008F0DCFAF8BDC0460004FF1F0E
:1037E000B064FF1F806FFF1F7C44FF1F4A0AFF1F4A
:1037F0003A07000080C3C9019A020000DC050000FE
:103800006A18000050C3000088130000F009FF1F71
:10381000204E00006509FF1F68100000C409000069
:1038200040420F0010270000FC00FF1FB91CFF1FC3
:103830000000FF1F0D2DFF1F9530FF1F2D2FFF1FB5
:103840007920FF1F6927FF1F9520FF1F4122FF1FBF
:103850000520FF1F8D29FF1F752AFF1F9519FF1FC8
:103860009928FF1FBD25FF1FC925FF1F051FFF1F2B
:10387000BD1FFF1F7D1EFF1FF0B502250124614BF8
:1038800091B01D700293604B604E1C70604F0393AB
:10389000336800212800FB7006F08EFE280006F039
:1038A00085FD0023984205D0FA78552A02D0332AA4
:1038B00000D09AE03360042006F0E6FF08F048FAF2
:1038C000FFF75CFE07F0FCFF1F2201240021514B93
:1038D00010AD1A70504B1C70504B1970504B19683A
:1038E0009143163A0A431A60602219689143403A9C
:1038F0000A431A6008F074F908F0F2F8494B984747
:10390000C120FF21484B80001A588A431A50C52213
:10391000920098588843BF390143995098584349B9
:1039200008408021C9010143802099509958C00561
:103930000902090A0143995080213D48490108F0D4
:1039400097F9032322003B49019400933A4808F079
:103950001FF82C22394905A808F04AFA05AC61780D
:103960002078023406F042FDA542F8D1344C354BA4
:10397000226803201A40A023DB0213432360802324
:1039800022689B041343236022682F4B1A40802334
:103990009B03134323602D4A2D4B934200D80120F3
:1039A00007F0EEFF07F0F4FE80232268DB041343E8
:1039B0002360029B187808F0C3F8039B1878C0B204
:1039C00008F0A6F808F004F82249042007F0E8FE01
:1039D00006F026FF00F040F800F030FE00F0D8FEC0
:1039E00000F018FA002011B0F0BD00932100194A30
:1039F000042008F0BDF88023DB059C62FFF768FD1A
:103A000059E7C0464A0AFF1F7C44FF1F34F00040BC
:103A10003C62FF1F480AFF1F490AFF1F680AFF1F79
:103A2000BCF00040E1A2000000E100E0FF00FFFF69
:103A30008044FF1F0457FF1F8054FF1F00BE00116A
:103A400014F00040FF7FF8FFFFFF9FFF0080FF1F83
:103A5000806FFF1F3B000108002210B511001120EC
:103A600007F0DEFE10BD0000F8B500230925374F32
:103A7000374C3B62E3681120AB43E36007F018FF6B
:103A8000112008F04DF9112007F092FE4023226822
:103A900080261343236080236268DB021343636044
:103AA000A3682C4A3343A360A36828001340A36093
:103AB0008023A2689B0113431022A360236C022180
:103AC00093432364236C0F3A1343236480235B01E5
:103AD0003B62226B204B1A402263626B1A40626386
:103AE000A26B1A40A263E26B1340E363E3681B4AD4
:103AF0001340E36006F07AFC2800012106F08AFDFD
:103B00008023174A9B00516C11200B43536408F02B
:103B10003FF8FD21134B144A89005A508023C720D7
:103B2000E26B5B031343E363E36880001D430F4BC9
:103B3000E56019580E4A1140802212020A431A50B9
:103B4000802292051A600B4B5E63F8BD00F00040C6
:103B50003CF00040FFFFDFFFEFFFEFFFFFFF7FFFC5
:103B6000003800400000FF1F5118FF1F00E100E077
:103B7000FF00FFFF00000540E12010B5C00407F082
:103B8000E7FE10BD70B52B4C238C002B2AD0FA22F7
:103B9000D200934201D2FFF7EFFF228A238C002A42
:103BA00021D1DA0023826382A382E38223836383A9
:103BB000A383E38322606260A260E2601E4D1F4A1D
:103BC0006420EB8093420AD8FA220020D20093426C
:103BD00005D91B4A0A21981807F042FEC0B20023FB
:103BE0002872238470BD0720E11CCA7F0132024085
:103BF000CA7705D10325201DC17F01312940C17736
:103C000008325200A352002321001A00088A013210
:103C10001B180231082AF9D1221DD27F9200A3502D
:103C2000626823689B18A2689B18E2689B185B096E
:103C30009BB2C3E77C61FF1F2462FF1FB70B00002C
:103C400030F8FFFF30B503A804880B20002C0ED1FC
:103C50004968074D08784978090201430A20A942BA
:103C600005D1012120001980024B1B7A137030BD51
:103C7000192A00002462FF1FF7B5150008AA16884C
:103C80004A680F4F14785278120222430A24BA422B
:103C900014D10122DBB2019200962A0007F010FD38
:103CA000041E0BD1074B1B68002B07D068782A78BD
:103CB0000002104342425041013098472000FEBDAF
:103CC00002290000A861FF1F30B501250379040017
:103CD000BFB02B4211D00A49408807F05DF8284256
:103CE0000BD0084B01A95B8D4D800B80064B002249
:103CF0001B7A60880B7104F041F93FB030BDC046BB
:103D0000A061FF1FB040FF1F2462FF1F10B50549CF
:103D1000054806F0F7FF0421044A054806F0B4FF01
:103D200010BDC046A061FF1FFFFF00002CBE0011A8
:103D3000B040FF1F10B5024804F0A2FF10BDC046FE
:103D4000C93C0011012303700B4B1A7A4270022206
:103D500082709A78C270DA780271032242711A79FD
:103D600082715A79C2710C2202729A794272DB799D
:103D700083720B207047C0462462FF1F022310B5D8
:103D80000370013B43700533837010330371443B70
:103D900043712A3383714433C37100230372064B8A
:103DA00004001B8843720A30FFF7CCFF831D0A30E2
:103DB000C0B2E37010BDC0462462FF1F10B51420CE
:103DC00007F006FF124B14220021186007F098FD3F
:103DD000002007F015FF012007F0C2FF022007F0C6
:103DE0008FFE032004F0F0F9042006F005FA052008
:103DF00003F02EFC062004F0FBF8072001F0A8FADF
:103E0000082006F021FF092001F082F810BDC0460D
:103E1000AC61FF1F07F05CFE012007F0A9FF07F06F
:103E200027FE0000094B10B50400984205D0012977
:103E300004D12000064906F065FF10BD0229FCD11F
:103E4000013904F0DBFE0028F3D0F6E7FEFF0000A6
:103E5000D261FF1F70B50D7A100004AA2C001688DD
:103E600010221440154220D1002E20D10A78022AB7
:103E700018D14A68517815780E4A090229439142AF
:103E800005D00D4A914209D01C800A2404E0142276
:103E90000A491A8007F0ACFF200070BD0C220849C7
:103EA0001A80F7E71C800124F6E70824F4E70B24C6
:103EB000F2E7C046F3FF0000F4FF00000843FF1FD5
:103EC00028BF001110B504000749084806F01AFF82
:103ED000074804F015FE0020E40704D50721054A31
:103EE000054806F0D1FE10BDD261FF1FFFFF0000A4
:103EF000253E001170BE0011F440FF1F00B50C4BB1
:103F0000BFB01A780B4902A800F0FCFC6B4680B2E7
:103F1000D880002809D06A46074B01A91B889380E6
:103F2000064B0022188804F029F83FB000BDC046B7
:103F3000B061FF1FB161FF1F4E41FF1F5842FF1FBD
:103F400000B50C4BBFB01A780B4902A801F05CFF1A
:103F50006B4680B2D880002809D06A46074B01A979
:103F60005B8D9380064B0022188804F007F83FB061
:103F700000BDC046DA61FF1FDB61FF1FF440FF1F79
:103F80005842FF1FF7B50E00377A1C0008AB11002E
:103F90003D001A8820231D401F423CD13378022B5C
:103FA0003BD173681F785B781B023B431E4FBB42BB
:103FB00008D01E4FBB4214D01D4DAB4221D00A2564
:103FC0002800FEBD002A2AD1142C2AD82200F0682D
:103FD00007F00EFF174B1C70012CF1D9FFF7B0FF53
:103FE000EEE7002A1BD1202C1BD82200F06807F036
:103FF000FFFE114B04211C70104B187807F090FD48
:10400000DEE7E3B20124009201940A00310007F0D8
:1040100057FB0500D4E70825D2E70125D0E70B259B
:10402000CEE70D25CCE7C046F3FF0000F4FF00000B
:1040300002290000DA61FF1FB061FF1F5C62FF1FF1
:10404000332310B5040003700A220749013007F03A
:10405000CFFE064B0F201B681A0AE37222731A0C5C
:104060001B0E6273A37310BD2462FF1F4C62FF1FFF
:1040700030B5012503790400BFB02B4213D00B49A2
:10408000408806F089FE28420DD06A46084B02A8F7
:104090001B889380FFF7D4FF6B46D880002260888E
:1040A00001A903F06BFF3FB030BDC046D261FF1FD6
:1040B0004E41FF1F10B5024804F0E2FD10BDC0469E
:1040C0007140001170B5160004AA148805AA15786D
:1040D0004A685078117800022A4A08438018052857
:1040E0004BD807F0CDFD03131E29343F0720042CC5
:1040F0000BD80522121BAA4200D92A0022491A8095
:104100003000091907F074FE002070BD0720112C43
:10411000FBD81222121BAA4200D92A001B491A807E
:10412000EEE707200E2CF0D80F22121BAA4200D96E
:104130002A0017491A80E3E70720032CE5D8042258
:10414000121BAA4200D92A0012491A80D8E7072078
:10415000032CDAD80422121BAA4200D92A000E49E5
:104160001A80CDE70720032CCFD80422121BAA42C5
:1041700000D92A0009491A80C2E700220A201A80C1
:10418000C3E7C046DCD5FFFFBBBE0011F861FF1FCF
:10419000ABBE0011A6BE0011A1BE00119CBE001155
:1041A00010B50D21024A034806F06EFD10BDC04651
:1041B00090BE00116441FF1F13B5104C0423217CF5
:1041C00001AA00F0ADF9002815D16B469A88236842
:1041D00052BA92B25343228909491B0C9B184B8057
:1041E0006B46DA88636852BA92B2534362891B0CF9
:1041F0009B188B8016BD0120FCE7C0460C62FF1F98
:104200002462FF1F13B5124C06236A46217C00F07E
:1042100087F9002819D16B461988236849BA89B2F1
:104220004B4321890B4A1B0C5B1853806B46D97892
:1042300003335B781B020B435BBA61689BB24B4351
:1042400061891B0C5B18938016BD0120FCE7C046FA
:104250000C62FF1F2462FF1F37B5174C07236A4605
:10426000217C00F05DF9002824D16B461B787F2B60
:1042700020D86B46DD78F0232A041B031A406B46D6
:104280009B880E495BBA9BB21A4323682D0953439E
:1042900022891B0C9B184B806B465A789B78120323
:1042A0001B011A4363682A43534362891B0C9B1802
:1042B0008B803EBD0120FCE70C62FF1F2462FF1FC4
:1042C0007FB50226154C0022217C03AB0096050029
:1042D00000F0F8F8002802D0012004B070BD0E23D1
:1042E000217C0122280000966B4400F0EBF80028A6
:1042F000F2D16B469A892368D2BA5343228908497E
:104300001B149B184B806B46DA89636852BA92B2D1
:10431000534362891B0C9B188B80DEE70C62FF1FE6
:104320002462FF1F70B5184C237C002B0FD0382B54
:104330000ED1164D280000F073F8CC23AC222800D3
:10434000217C9B0100F027F9280000F0A7F870BD40
:10435000E3890F4A934209D10C4D280000F060F820
:1043600000222800217C00F005F9EDE7094A93427C
:10437000EDD1064D280000F053F890222800217C52
:10438000920100F026F9DFE70C62FF1F3C42FF1F9D
:10439000830500008320000070B5144C237C002BA3
:1043A0001FD06369002B1CD0114D280000F038F895
:1043B0006369280098470400280000F06FF8002C7B
:1043C00010D10C4B0422995E002905DA9C801A88D2
:1043D00001321A80200070BD074A9142F7DD9A80B1
:1043E000F5E70124FEF784FEF4E7C0460C62FF1FE8
:1043F0003C42FF1F2462FF1F0F27000010B58024DE
:10440000064AA4001168436B234205D113685B1A66
:10441000032BF8D9012010BD0020FCE76008FF1F26
:1044200070B5C17905000C00631E9C411A4BE40273
:10443000E41849000460C9B2007906F021F9E9796D
:10444000687949000131C9B206F01AF9E8790930F2
:10445000C0B207F0ADF90023E36661332360AA79A7
:104460005B3B002A0ED022689A43023B1343236031
:104470000A23E3610733236200232363A363013329
:10448000E36370BD22689A430223134323604623EB
:1044900063610633A361EFE70050004070B500256B
:1044A00004000368DD66C0790930C0B207F000FA85
:1044B0002900207906F080F82900607906F07CF860
:1044C00070BD0000F8B51E0006AB1D78002304681F
:1044D0001700E366616007F0E3FB01238022E366D7
:1044E0002B0027615200013B08D207F0F1F90820A8
:1044F0000A4A1168002D03D12800F8BD2261F2E7B5
:10450000236F034203D02369013D337001361368E2
:104510005B1A032BEED90125EEE7C0466008FF1FAA
:1045200070B51C00002305681600EB66696007F093
:10453000B7FB01238022EB6623005200013B08D227
:1045400007F0C6F908200A4A1168002C03D12000A0
:1045500070BD2A61F2E72B6F034203D02B69013C47
:104560003370013613685B1A032BEED90124EEE792
:104570006008FF1F002370B504681500E3666160E2
:1045800007F08EFB0123E366256107F0A1F9200007
:10459000FFF734FF70BD70B51D00002304681600DE
:1045A000E366616007F07CFB0123E36626610F335D
:1045B000626B1A42FCD02B0A23611023626B1A42F1
:1045C000FCD0EDB2256107F083F92000FFF716FF5C
:1045D00070BD002370B504681500E366616007F0E4
:1045E0005FFB0123E3662B0A23611023626B1A42EF
:1045F000FCD0EDB2256107F06BF92000FFF7FEFE5D
:1046000070BD70B51E00002305681400EB6669607C
:1046100007F046FB0123A619EB660F33B44205D120
:1046200007F056F92800FFF7E9FE70BD21782961EF
:10463000696B1942FCD00134F0E7000010B5084C5A
:10464000E368002B08D18022064B52021B689B189E
:104650006360054B1B68236007F0E2FAA06010BDA1
:104660004C62FF1FC8F00040CCF0004070B5184A03
:10467000936A916A9942FBD116498A689A421FD37C
:104680009A1A8B60144B0126186893B2D202D20E8C
:104690004343424300204C681B0A1B1912029B181B
:1046A0000E4C0A684B60551CA3420CD8002801D060
:1046B0004B600A600A4A136008680A4B186070BDB4
:1046C000581E821ADDE7084A30009B182A00EAE7E4
:1046D00000F000404C62FF1F140AFF1F40420F0011
:1046E000C8F00040CCF00040C0BDF0FF70B51F4CDA
:1046F00023793F2B01D93F2323711D4B22791A7057
:104700001878C0B207F0C4FA18231A491A4A0B8065
:104710001A4913800B805380A379194980200B809C
:104720000C21938001334B43164D191C0001834229
:1047300000D9011C2980D1806379002B01D101337C
:104740006371237A012B01D8022323726279237AC1
:104750000D4853430A21584307F082F80B4D286057
:10476000E379052B01D81023E37170BD4062FF1F70
:10477000480AFF1F5642FF1F2844FF1F5442FF1FD5
:104780005242FF1F5042FF1F710200003062FF1FA4
:10479000F8B520210020FEF763FE114C011E114DDB
:1047A00009D10C22104BC1CBC1C4280007F0A8F8D6
:1047B000FFF79CFFF8BD0C2220000C49FEF724FEF9
:1047C0000C2802D0084B43CB43C40C2228000849D4
:1047D000FEF71AFE0C28EBD00C220021E5E7C046BC
:1047E0004062FF1F0C62FF1F1CBF0011FC0C000089
:1047F000F50C0000F0B51D4C8022A5440400882073
:1048000069465201400507F04BF9902212016A44B3
:104810001300200032C832C316C816C38023144CBC
:10482000144FA6689B033343A3603B6006F0C8FFA8
:104830008823A0685B05C01807F072F8002588235C
:1048400029008022A0685B05C01840196944520005
:1048500007F0EEF880230135FF355B019D42EED174
:10486000A6603E60044B9D44F0BDC046FCEFFFFFD8
:104870009843FF1F9808FF1F04100000F0B50400C4
:1048800087B0002825D0684607F002F91B4C0228A3
:1048900006D106226946200006F0BAFF002816D08D
:1048A0006946002301250F262F00E25C0133100921
:1048B0001030874038002F00324097403A000243C2
:1048C0004A610439062BEFD16846FFF793FF07B022
:1048D000F0BD182269460A4807F0E2F86A46A300CC
:1048E000D358013305D01822FF21684607F008F895
:1048F000EAE70134062CF1D1E9E7C0466509FF1F5C
:1049000000090011F0B5002504000E0085B0AA4290
:1049100000D186E04B1C087801934B788978377971
:1049200009021943F3783F061B040B431F43039707
:1049300020706570252800D196E033D8112813D84F
:1049400007F04EFA69003201320132013201AA0049
:10495000B800B100320132013201320132013201BC
:10496000320132010C012C01232800D1E5E0DB28C3
:1049700000D03BE1042A00D8B1E01025052A05D07B
:10498000551F2A003800711D07F032FA0522310048
:10499000200007F02DFA2A003900601D07F028FAE0
:1049A00005353EE0562859D010D8332800D1A7E06D
:1049B000552839D02628DAD1A24B29001322180015
:1049C0001D0006F09DFFFEF793FB5CE0712800D10F
:1049D00077E0722800D189E0602800D195E0DC28DA
:1049E000C5D1022A00D87AE07378BFB26370B37879
:1049F000A370032A05D0033A390092B2F01CFEF7E7
:104A00003DFC10223900E01CFEF7FEFCC51C00280E
:104A100007DA607070E00C2220008B4907F0E8F99B
:104A20000C25280005B0F0BD013A884D0C2A13D89A
:104A3000002A0AD02800019907F0DAF9FFF756FE9C
:104A40000C2228008249FEF719FC29000C22601C68
:104A500007F0CEF90D25E4E70C22EBE77B4D7D4B0B
:104A60002A0043CB43C2E9E7013A764D0C2A11D81C
:104A7000002A08D00199280007F0BAF90C22280072
:104A80007549FEF7FBFB29001322601C07F0B0F903
:104A90001425C6E70C22EDE706227049601C07F0DA
:104AA000A7F90625BDE712226D49601C07F0A0F9A1
:104AB0001325B6E708226B49601C07F099F9092510
:104AC000AFE7012A0ED07178F02908D8664D288802
:104AD00001F0F6FD654B2A885200D35A00E0FF230F
:104AE000637009E0604A614B1288F5E7604B012A68
:104AF00004D072789A706270022592E79B78EFE793
:104B00002000FFF79DFA05008BE7013A584B594DFD
:104B1000082A0DD8002A0DD00121280059700199CA
:104B200007F066F901F088F808222900601CC4E744
:104B30000822F1E700225A70F6E7042A04D94E4D04
:104B40002F6007F06DF8A860FFF790FD0422039036
:104B500003A9601C07F04CF9052562E7474D062ABA
:104B600015D906222800019906F052FE00280ED021
:104B700006220199280007F03BF906224049280047
:104B8000FEF77CFB01233A4A91780B43937029008E
:104B90000622601C07F02CF9072542E7012A9ED067
:104BA0007078FFF76BFEA7E7012800D0DFE6931EC1
:104BB000344F132B06D87378002B0BD100F016F965
:104BC00000F04CF9304B39001D78601C6A1E07F06C
:104BD0000FF926E7551E2A000199380007F008F959
:104BE00038002A49AAB2FEF749FBE9E7DA281DD1C5
:104BF000042A00D873E7082A15D9B37972791B0201
:104C00001343F27912041A43337A1B0613433B60B1
:104C10003B68052231002000039307F0E9F80422E5
:104C2000601D03A949E7FE236370F1E7DE2800D089
:104C300055E7511E012A01D10025F2E6019800F046
:104C4000E1FFF9E70C62FF1F28BF00114062FF1F60
:104C5000FC0C00001CBF0011F50C00001862FF1FC7
:104C6000F861FF1F9C43FF1F5842FF1FB464FF1FE2
:104C70003C62FF1FF542FF1F4C62FF1F6509FF1FCB
:104C8000ADAC00003D64FF1F3B64FF1FAEDE0000C3
:104C900070477047020010B5094B0A32094C92B2B6
:104CA000DA815A8298811882207802F06FFB042200
:104CB000054B012120781A7006F032FF10BDC04666
:104CC0002643FF1F8664FF1F8564FF1F013870B5F0
:104CD000042809D806F0D4FF030928081200234B42
:104CE0000221187806F01CFF70BD204B08211878AF
:104CF00006F0A6FE00221E4B1A72F5E78022002461
:104D00001B4B1A4D52001A8108211A682878DC7250
:104D100006F046FE2100287806F0FAFD012000F09A
:104D200077FE00F089FFDFE7104B0821187806F0C6
:104D300087FE1048FFF722F80F4B104A9B7900209E
:104D400093800F4A13808022094B5200D8721A8137
:104D500000F05EFE00F070FF0A4B9B78002BC3D082
:104D6000094A136006F074FEBEE7C0465C62FF1F8E
:104D70003062FF1F6142FF1F4062FF1F2844FF1F78
:104D80005242FF1F3C62FF1F34F0004010B5002963
:104D90000BD1022809D1054B1B78002B05D0262208
:104DA000034B04485A72FFF775FF10BD5E64FF1F86
:104DB0003062FF1FC40900000300F0B50A4D8E18D1
:104DC000B14202D152008018F0BD0C782F6824093E
:104DD0003C5D0F271C700C7801313C402F683C5D16
:104DE0005C700233ECE7C0464C42FF1F0E22124BB0
:104DF00010B51A700D23114C11492370093A043B68
:104E00001048637006F0F4FF2D2301220E490F486D
:104E1000E371FFF7D1FF01220D49FFF7CDFF01221A
:104E20000C49FFF7C9FF030000200B49020018706E
:104E3000FEF724FA10BDC0465A64FF1F3B64FF1FF3
:104E4000BBBE00113D64FF1F6709FF1F4364FF1FC6
:104E50006609FF1F6509FF1FAEDE000070B5134C29
:104E6000142220001249FEF7CFFA431E114D132BD6
:104E700019D8AB78002B16D0431C2B7009236B700C
:104E800000230019037028780B4B01302900C0B2B1
:104E9000187006F005FD297822000139C9B20020FA
:104EA00005F010FE70BDFFF7A1FFECE73D64FF1FAA
:104EB000AEDE00003B64FF1F5A64FF1F10B5114BAC
:104EC0001A781870002A0ED000280BD10E4B1A78D1
:104ED000062A07D85423D340DB0703D50B4B187899
:104EE00002F054FA10BD0028FCD0074B1B78012BB0
:104EF00002D0033B022BF5D8044B0121187806F0B1
:104F00000FFEEFE75E64FF1F8564FF1F8664FF1FCF
:104F100070B54A4E4A4A4B493070022005F05EFC9B
:104F200000F00EFFFEF7E4F806F0E2FC032246492B
:104F30004648FFF741FF2D24030004221C7044491A
:104F40000130FFF739FF30230470424D424C43706B
:104F500083702E3B062220004049EB87FEF754FA6F
:104F6000062813D0200006F093FD022809D0032163
:104F7000200006F03DFD8D23E3706E3B2371193355
:104F80006371062220003549FEF778F9344B1B681F
:104F9000FC335C64FFF762FF0020FFF78FFF314CAA
:104FA000314A0121314B1278207802F0B1F9304AB0
:104FB000304B12780021207802F0AAF901222E4B02
:104FC0001A702E4BDB78552B31D12D4B3B325A7258
:104FD0002C4B2D4AAB81EA812B826A8220213078CA
:104FE00006F036FC0120404205F0B8FD01204042A9
:104FF00005F054FEFFF7D4F8FEF788FE00F0B2FC8F
:1050000001204042FEF75EFF012006F0F9FCF0208F
:1050100001F03AFB0121307806F082FD307802F091
:1050200011FB1A4806F01CFDFEF71EFD70BD642240
:10503000174B5B7953431A000A32CBE75C62FF1FC0
:105040008D4D0011914C00119C43FF1FF861FF1F13
:105050001862FF1F2643FF1F6509FF1FADAC00004C
:10506000B064FF1F8664FF1F8042FF1F6142FF1F65
:105070005A64FF1F3B64FF1F2C64FF1F3C62FF1F2D
:105080003062FF1FC4090000CE0900005E62FF1FEE
:105090004062FF1FF8B50A0020230D001A40194294
:1050A00063D05E4B1B78002B5CD0FFF7DFFA5C4BC4
:1050B0005C4C5D4E99686268737A8A1ADB039A4287
:1050C00002D36160FEF7D0FC327A217A531EDBB244
:1050D000994205D1FFF726F9002000F0E9FD15E01F
:1050E0009142F9D300272772FFF756F9A37ABB4202
:1050F00002D0A772FEF746FD012000F0D9FD4B4F0C
:105100003800FEF73BFE390006F0D2FD637A002B33
:1051100025D0013BDBB26372002B20D1444BDB78FE
:10512000552B01D106F094FCE37A002B12D000231A
:10513000A27AE3729A4202D0A372FEF723FD3D4A9F
:105140003A4F1388380001331380FEF717FE3900F9
:1051500006F0AEFD642370795843FFF79BFD237A78
:105160000133237220206840F8BD0BB2002B0ADA0D
:10517000314B187806F0A4FC002801D006F038FB6B
:1051800080200002EFE70224214206D0254B0120B7
:105190001A72FFF793FE2000E5E70B071ED5FFF715
:1051A00065FA1F4B1F49204C98684A68637A821A37
:1051B000DB039A4202D34860FEF756FCFFF7ECF897
:1051C000FFF7B0F8012000F073FD00F0E5FB236865
:1051D000DB0701D5FEF76EFF0820C4E7CB0609D533
:1051E000FEF7D0FC0D4B1B78002B01D1FEF7A2FD82
:1051F0001020B8E70124214207D0104800F06CF8D5
:1052000006F0F6FC00F034FDC5E704240800204059
:105210002142A9D0FEF772FEBDE7C0465E64FF1FC3
:105220004C62FF1F3062FF1F4062FF1F6142FF1F81
:105230003C62FF1F2462FF1F5C62FF1F4442FF1F8E
:10524000F0B51B4B1B4F1B883A8804001A4E1B4DB0
:1052500085B09A420DD832889A420AD3184B1A88E0
:105260002B889A4205D1174A174B12881B889A42FD
:105270001BD0052001F05EFA3B8802AA1380338818
:10528000019053802B88114D93800F4B02A91B88EE
:10529000D3800F4B2A78188802F07AFF0D4B082133
:1052A0002878019A1C7006F0E3FA05B0F0BDC046FC
:1052B0002A64FF1F5642FF1F5442FF1F5242FF1F26
:1052C0002864FF1F2664FF1F5042FF1F8664FF1FD4
:1052D0005842FF1F2464FF1F13B50C4B1C78002C91
:1052E00011D1002801D00A4B18600A4A0A4B1178E4
:1052F0000A4A10780A4A01920A4A0092002205F0EE
:10530000D9FA200016BD1124FBE7C0468564FF1FB3
:105310002064FF1F8464FF1F7464FF1F8664FF1FE7
:105320006064FF1F6464FF1F10B5064B12201B78DA
:10533000052B06D1044B13221988044B187801F071
:10534000D5FB10BD8564FF1F5842FF1F8664FF1FF9
:1053500010B500240122114B52421870104B1C70E2
:10536000104B1A8002F06EF904220F4B21001A70C4
:105370000E480C3206F0ECFB102221000C4806F01F
:10538000E7FB07220B4B1C600B4B1C700B4B1C707C
:105390000B4B1A700B4B1C7010BDC0468664FF1F70
:1053A0008564FF1F5842FF1F8464FF1F7464FF1F42
:1053B0006464FF1F6064FF1F3A64FF1F3964FF1FAE
:1053C0005A42FF1F3864FF1FF8B5174C06002578B6
:1053D00006A814240078052D23D1B41F134FA5B2BD
:1053E0001824BD421DD88D1FADB2BD4219D8FA2573
:1053F0006D00AA4215D21D000D4F0A3DADB2BD424F
:105400000FD80C4C26800C4C21800C4900240A80BB
:105410000B4A1380FFF714FF0A4B0421187806F09B
:105420000FFB2000F8BDC0468564FF1F790C00000B
:10543000750C00005642FF1F5442FF1F5242FF1FCF
:105440005042FF1F8664FF1FF0B50BB20D0089B0FC
:10545000002B00DB70E1A44E307806F031FB041E17
:1054600050D00378A22B00D122E1D02B1AD0912B5F
:1054700045D143780E2B42D19C4B82889A423ED133
:105480009B4A83681278052A39D1032018567F2851
:1054900035D0984B1B68002B31D05B68002B2ED089
:1054A00098472CE08078072829D806F0E9FB0428E3
:1054B000183F3F74A8D86378002B0CD101218C4B86
:1054C00019708D4B1A78002A5BD08C4B307801F024
:1054D0001FFF002855D00722854B1A7051E06178D4
:1054E0000029F8D1E378002B11D0854A854B12783A
:1054F000307801F00DFF60706378002BEBD1200055
:1055000006F076F980200002684009B0F0BD784BC3
:105510001B78022BF3D00121307806F049FC0028DB
:10552000EAD10121307806F0FBFAE5E76378002B39
:10553000D1D16F4F032807D13B78052B02D101331E
:105540003B701EE00223FBE76F4B1A886F4B029300
:10555000002A0BD01B78002B03D00121307806F0F5
:1055600087F93B78062B04D1013BE9E7029B1A70CF
:10557000F7E7042B41D10121029B3078197006F026
:10558000CFFA5C4B1B68002BB9D01B68002BB6D040
:10559000574A107884E76378554F002B27D10622AD
:1055A000211D5B4806F024FC62895A4B5A491A8037
:1055B000A2895A4B1A80E3890B800521397058491A
:1055C0000A80584A1380228A574B1A80574B1B78FF
:1055D000012B09D11F2001F0ADF8FA2292004243BD
:1055E0000421307806F044F90022484B75E7312B4E
:1055F00000D070E70022454B1A700323A0E7062273
:105600000021434806F0A4FA0023454A04211380F0
:10561000444A30781380444A138006F011FA082176
:10562000307806F00DFAA379083B5A425341304ACC
:1056300003331370304B1B78002B06D0334B30787C
:105640001A78002A06D001F0A1FE0122314B524205
:105650001A8096E70121197006F062FAF5E7082131
:10566000307806F0EDF96378002B00D047E72C4B3B
:105670002D4F0293E388029A04211380294B30783E
:1056800003932389039A138063893B8006F090FB80
:10569000002800D033E7264B1B68002B00D12EE7F3
:1056A000039902983A88098800881B68984726E77A
:1056B0004379132B00D022E70389012B0AD11D4B1C
:1056C0001B78022B06D10821307806F0B9F9FFF7D4
:1056D0002BFE14E7052001F02DF808210200307898
:1056E00006F0C6F80BE7C0468664FF1F05140000ED
:1056F0008564FF1F2064FF1F8042FF1F6142FF1F60
:105700005A64FF1F3B64FF1F5C64FF1F5E64FF1F42
:105710002D64FF1F5842FF1F3464FF1F3664FF1FB4
:105720002A64FF1F2864FF1F2664FF1F2C64FF1FCD
:105730001C64FF1F2464FF1F8020C001014200D0B1
:10574000E2E6CB0731D5324B1B78002B1DD0314E12
:1057500005AC3378052B1AD1023B23702E4B210068
:105760001B7823722D4B1B7863722D4B187801F038
:1057700073FD002809D007202A4B30701B68002BCE
:1057800003D01B68002B00D098470120BCE60E20F8
:10579000254B06221B7825492370254B1B78637007
:1057A00002ABC01806F024FBD8E70223080018401B
:1057B000194209D0174B1B78052B03D11D4B1888B4
:1057C00006F066F802209FE60424214203D0FFF78A
:1057D00037FD200098E6082308001840194200D140
:1057E00093E6154B1C78012C03D0022C0DD0082019
:1057F0008AE6124B124A134913481B8812880988FB
:1058000000880094FFF7E0FDF1E7FFF78DFDEEE77C
:105810005E64FF1F8564FF1F5A42FF1F3864FF1F2D
:105820008664FF1F2064FF1F3A64FF1F5B42FF1F57
:105830003964FF1F5842FF1F2464FF1F5042FF1F9F
:105840005242FF1F5442FF1F5642FF1F10B502A8CD
:1058500004880B20002C10D1496808784978090287
:1058600001430C48814209D1022119800A4B598811
:105870001170DB7800205BB2537010BD074C0A201A
:10588000A142FAD102211980034B998811705B79EA
:10589000F0E7C0466E2A00002462FF1F6F2A000056
:1058A000F7B5150008AA16884A680F4F1478527881
:1058B000120222430A24BA4214D10122DBB201921D
:1058C00000962A0005F0FCFE041E0BD1074B1B6856
:1058D000002B07D068782A780002104342425041DA
:1058E000013098472000FEBD022900009864FF1F88
:1058F00030B5012503790400BFB02B4225D01449EF
:10590000408805F049FA28420CD0124B01A95B8D62
:1059100000220B8002234B800F4B5B888B806088BA
:1059200002F02CFB0D49608805F036FAC0070CD553
:105930000B4B01A91B8800220B8002234B80064BD6
:105940009B888B80608802F019FB3FB030BDC04659
:105950009064FF1F8442FF1F2462FF1F8864FF1FA3
:10596000DE42FF1F10B5074C0749200005F0CAF9B9
:105970002000064905F0C6F90721054A054805F04B
:1059800083F910BDFFFF00009064FF1F8864FF1FB4
:1059900048BF00118442FF1F10B5024803F070F9A0
:1059A00010BDC046F1580011082110B50E240A4A56
:1059B000C307DB170B405179A1430B4353710223FB
:1059C000184202D051790B4353710423184202D07C
:1059D00051790B43537110BDF542FF1F0A2110B5D9
:1059E0000F240A4AC307DB170B401178A1430B436E
:1059F0001370830703D5062311780B4313704007F8
:105A000003D5012311780B43137010BDF542FF1F1E
:105A100010B5054B102419780A00A243002801D0C4
:105A200022000A431A7010BDF542FF1F662110B50F
:105A30002024134BDA788A431979DA70A1432419A8
:105A40000C431C71542812D96020014319710421A0
:105A50000A43DA700222D9780A43DA702022D97810
:105A60000A43DA704022D9780A43DA7007E0442802
:105A7000EDD83428EED82428F0D81428F2D810BD58
:105A8000F542FF1FF8B50E23384C050062792679E0
:105A90001A4011339E43364B62712671984204DDE1
:105AA0006E23E3716C3BA371F8BD324B984203DA6D
:105AB0001A23E3711C33F6E700232F49A371E37126
:105AC00083B259182D4889B2814224D9681D0A2110
:105AD00000B205F0C5FE2A4B00B29D4244DC050031
:105AE0006421280005F0BCFE0A2100B205F0E0FFA9
:105AF000244F09B2E2797B5C1343E3710A21280049
:105B000005F0AEFE0A2100B205F0D2FF1D4F09B22A
:105B10007B5CA2790EE001210A436271002D1CDA40
:105B20005B421DB20423A371A379632DD8DCFA2252
:105B3000092DE3DC1343A3710A21280005F0B8FF07
:105B40000F22114F09B27B5C1A4016431F22934368
:105B50006279267113436371A6E7FA239B009D4285
:105B6000E2DB0123E371BBE70500FAE7F542FF1F23
:105B70001B4E00001DFCFFFFCB070000960F00002E
:105B80000A27000092BF001182BF001170B51B4DA3
:105B900004002B7900290DD0802213432B71632C34
:105BA0000BDD76236A7813436B704023AA78134386
:105BB000AB7070BD7F221340F0E72300093306DA93
:105BC00058236A7813436B70AA786C23EFE70C4E66
:105BD000002C0ADA2023644224B26B700A212000D0
:105BE00005F066FF09B2735CE2E7092CF6DD0A21D5
:105BF000200005F035FE00B2335CEEE7F542FF1FF2
:105C000072BF0011F8B50A4F05003B780E00002B5B
:105C10000CD0084C2000FEF703FC33002A002000C3
:105C20003978FEF7EEFC2000FEF738FCF8BDC046E0
:105C3000A564FF1F0043FF1F70B50A4E0A4D0822DE
:105C40003100280005F0E4FD002809D0074C3100A0
:105C50000822280006F0CCF809212000FFF7D2FF27
:105C600070BDC046F542FF1F9D64FF1F9C64FF1F6F
:105C7000102110B50D4B1A780A401A70DA78563197
:105C80000A40DA70602219791140223ADA71083A32
:105C90009A71AA325A71DF3A0A431A716B225A700A
:105CA0000C3A9A70FFF7C8FF10BDC046F542FF1FBF
:105CB00010B5002832D01E4C0223E05E1D4B1B683D
:105CC0005B062CD509233221584305F0C9FD41302C
:105CD000FF3000B2FFF7D6FE0520FFF765FE042275
:105CE000A35E154A6320934205DC32331800642119
:105CF00005F0B6FD00B20121FFF748FF207AFFF75B
:105D000095FE0020FFF76AFE0C4B187805384342D9
:105D10005841C0B2FFF77CFEFFF78EFF10BD0A218D
:105D2000053005F09DFD00B2FFF7ACFE0320D4E77F
:105D30002462FF1F4062FF1FDD2600008564FF1FF5
:105D400070B500250A4C2000A571FEF769FB1023F1
:105D50003E212000074AFEF754FCA84200D13E3500
:105D6000054B20001D70FEF799FB0123A37170BD48
:105D70000043FF1F62BF0011A564FF1F0200F0B5C2
:105D800001270A480A4E51188B1A002B00DCF0BD7F
:105D9000082415784308684038404000805B013C87
:105DA00058406D08002CF5D10132EDE7FFFF0000EF
:105DB000A2BF0011F0B500250F269D4200DBF0BD0B
:105DC0004C5D070944403440A400A0580135784098
:105DD000F3E70000F0B589B06A460D000B000F270D
:105DE000110010351C780133260024093E4016703E
:105DF00054700232AB42F5D12023024AFFF7DAFF9A
:105E000009B0F0BDA8BF0011F0B54E780B7889B08D
:105E100036020C00170001901E43012A61D9954BF0
:105E20009E4200D877E001339E421CD1062A17D14A
:105E3000CA788B7812021A430B791B0413434A79F0
:105E400012061A438C4B5A6100221A705A808B4AF0
:105E50005A608B4A9A608B4ADA60002009B0F0BD24
:105E600088225205EEE7884B9E423CD182498B78CE
:105E7000002B00D0F6E00C2A31D10F22A3789343F7
:105E8000E278120213432279120413436279120654
:105E900013434B60E279A07912020243207A000496
:105EA0001043627A12060243CA60E27AA07A1202B2
:105EB000024376484A81834208D804236E4914225B
:105EC00001980B7005F094FF1420C7E71201D21857
:105ED00089235B059A42F0D801238B70BDE7022A23
:105EE000FAD00523EAE76A4A01239642E6D1FFF792
:105EF0001BFA052F0CD9E378A2781B0213432279F1
:105F000012041A4363791B061343624A0393136016
:105F100005F09EFDA1E7584D2B78002B9DD1AB7865
:105F2000002B00D1A0E02B8901339BB20093B34238
:105F300000D091E0132AD4D9CF7C8B7C3F02122170
:105F400020001F43FFF71AFF874200D08EE0002E8B
:105F50003DD1E378A2781B0213432279E968120449
:105F60001A4363791B06134303930A228B4212D10F
:105F7000FF23A370E370237163716B89002B09D138
:105F8000E37B227C1B0212041343A27B13431B09F5
:105F900001336B8100226B89002B8ED0002A67D1E0
:105FA000686837013818000B6B690003039098424A
:105FB00005D9686105F0B4FCEB780133EB706868D3
:105FC0001022A11C381805F033FD2E8145E76F899A
:105FD000009A7B1E9BB293423AD1E278A3781202D8
:105FE0001A43237905A81B04134362796C681206CF
:105FF0001A43EB6800920392211D0C22049305F0D2
:10600000F7FE0120260004A940421036FFF7E2FE09
:10601000013F012F17D1009A0B232861824200D043
:106020004CE704221C49200005F002FD042203A9CC
:10603000686805F035FDE968039AFF23914200D1B5
:106040003CE7F73B3AE73100FFF7C4FE1036DFE7E5
:106050000923B742A4D831E7009BB34200D9FCE63C
:1060600007232BE7022329E7032327E7062325E756
:106070000A2323E7FFFE00000843FF1F0000011171
:10608000FFFF00005048593601FF0000FFFF0011DC
:1060900002FF000034F000401443FF1F10B5034C12
:1060A0000B000122210000F06BFA10BD5D620011AF
:1060B0000B8870B506000D000224162B11D92B0099
:1060C0000322094900F05CFA041E0AD1074B2A8812
:1060D0001B88191C934200D9111C300089B200F0B2
:1060E000EFFA200070BDC04689620011B664FF1F40
:1060F00010B54A780400013A0B000220012A07D8A3
:106100000A78002A04D005222000024900F038FA5B
:1061100010BDC046B76200110A7810B50B0004002C
:106120000220002A04D007222000024900F028FAA9
:1061300010BDC046636300110A7810B50B0004005F
:106140000220002A04D009222000024900F018FA97
:1061500010BDC046C963001110B5034C0B000B22E3
:10616000210000F00DFA10BDF963001110B5034CC9
:106170000B000D22210000F003FA10BD6B6400112A
:1061800010B5034C0B000F22210000F0F9F910BDEF
:10619000C56400110A7810B50B0004000220002A23
:1061A00004D011222000024900F0EAF910BDC046D7
:1061B000D5640011002310B51322190000F0E0F996
:1061C00010BD000010B5034C0B001722210000F099
:1061D000D7F910BD27650011002310B51922190049
:1061E00000F0CEF910BD000010B5034C0B001B22CF
:1061F000210000F0C5F910BD61650011F7B5848973
:106200000D0006000121002C22D000238268D35605
:106210001778002B1EDA0C2C1AD90C3CA4B21319D7
:1062200040880093230002F086FE431E984101300F
:106230007B06DB0F6B703F23013C1F40A4B228702C
:10624000AF70AC80002C07D0B3680133AB60002185
:106250000800FEBD0020EBE7AC60F8E70B780370A8
:106260004B8843704B881B0A83700B79C3700420E2
:1062700070470420022B06D10020537811781B02AE
:10628000009A0B43138070470B8803700B881B0A1E
:106290004370022070470420009983420AD153784A
:1062A00010781B0203430B80D37890781B020343C2
:1062B00000204B807047F8B50D004B780124002179
:1062C000461C03702B788B4201D82000F8BD6B78F8
:1062D000B01C4F1C012B10D1890069184B88022279
:1062E00033704B88B9001B0A7370691805F0E8FC1D
:1062F00004360434A4B2F9B2E4E7122359436B180C
:106300005A88043132705B8810221B0A7370691836
:1063100005F0D6FC12361234ECE770B5049D14007B
:106320001E00052B01D8042070BD637812781B0273
:1063300013432B80E378A2781B02134302226B8065
:106340002A71211D681D063E05F0BAFCB2B22A81F1
:10635000E92AE8D82800A11D0A3005F0B1FC002088
:10636000E2E7002310B50A789A4201D8900010BDE8
:106370009A008A185488013304705488DBB2240AC6
:106380004470948884709288120AC2700430EAE7DC
:1063900010B51100029C062B04D004201022142BEF
:1063A00001D010BD022222714B7808781B020343F2
:1063B0002380CB7888781B02034363800431601DFF
:1063C00005F07EFC0020ECE710B50C788B780431EA
:1063D0005C43E4B203702200013005F071FC601CE4
:1063E00010BD0420022B06D10020537811781B0227
:1063F000009A0B431380704710B50C000A880231D5
:1064000005F05EFC208810BD70B504000D000498F6
:106410001100012B01D8042070BD167852781202A9
:10642000324302800200F13255701470E125002CD5
:1064300000D10C35023B9AB24280AA42EBD802311D
:10644000043005F03DFC0020E6E70420009983427B
:106450000AD1537810781B0203430B80D3789078CD
:106460001B02034300204B80704710B50C000A88C4
:10647000023105F025FC208810BD000070B5012117
:106480001E000420049C0E400B4218D1CB40DDB20C
:106490008D4214D90A49DBB2098899420FD32300EF
:1064A000EE331D703300580011184978165C09024C
:1064B000314301332152D9B28D42F4D8002070BD4E
:1064C0002043FF1F10B50C000A88023105F0F8FBCD
:1064D000208810BD10B50C788B7804315C43E4B291
:1064E00003702200013005F0EBFB601C10BD10B5FD
:1064F00011000298032B01D8042010BD14785278A3
:10650000043B120222430280CA788C781202224392
:1065100042809AB28280EB2AEED80431063005F030
:10652000CFFB0020E9E710B50C000B8803700B8847
:106530001B0A43704B8883704B881B0AC3708A8880
:106540000430063105F0BCFBA088043080B210BDD9
:106550000420012B03D100201378009A1370704798
:1065600010B50C000B8803700B881B0A43704A8817
:106570000230043105F0A4FB6088023080B210BD07
:10658000F0B589B003931E4B029242000700D05A27
:10659000019102F020F81325061E2DD0029B012444
:1065A0000370019B002B04D0001903999847001930
:1065B00084B26B461B7A5BB2002B0FDA10213800D5
:1065C00002F01CFB1925002813D130003219E1B26A
:1065D00002F066FC051E0CD10C34A4B2042304AAFC
:1065E000380005A993800696948101F0AFFD051E41
:1065F00002D0300005F07CFA280009B0F0BDC0469A
:10660000B464FF1F70B505000C0000280CD00020FA
:10661000814209D010222000044905F051FB0120DD
:106620002B7823736B78637370BDC046E8BF00118D
:10663000F0B506000D0017001C0085B002291BD024
:106640000020102907D1022B07D0102B03D115E011
:106650000020102C08D005B0F0BD69463800FFF7C7
:10666000D1FF2A0069460BE069463000FFF7CAFFF8
:1066700022006946380004E0022BE9D12A003900E3
:10668000300005F08DFAE6E7031CF02800D9F0236E
:10669000032008499AB2013A0B80D31703400649F8
:1066A0009B189B100B80D30F04499B185B100B8029
:1066B0007047C0462443FF1F2243FF1F2043FF1F94
:1066C000034B1B888B4202D3024B4000C1527047E0
:1066D0002443FF1FB464FF1F014B4000185A70474A
:1066E000B464FF1F1722014B1A807047B464FF1F68
:1066F00070B505000E2005F06BFB041E13D0D023EF
:10670000037000230622837007494570033005F0AB
:10671000D7FA064B2100DA8A62811B7E2373044B71
:10672000187805F05DF870BDD064FF1FC064FF1FCE
:106730007443FF1F262803D8024B4000C05A7047FD
:106740000148FCE72643FF1FFFFF000070B506006D
:106750000C00094D1C220021280005F0F9F9074B17
:106760001E70074B1C7005F053FA0123002801D05E
:10677000002312202B7070BDC064FF1F7443FF1FE5
:10678000E164FF1F70B505000D4C0800E260A160D8
:1067900010220021656005F0CBF9012803D11021FA
:1067A000A06802F058FD10220021280005F0C0F971
:1067B000012803D11021606802F04DFD70BDC04674
:1067C000C064FF1F70B5041E05D1002903D0062246
:1067D0000D4805F075FA0D4B1D78012D11D1002CD7
:1067E00005D102221A7005F0BBF9280070BD002205
:1067F0001A70074B1B78FF2BF7D02000FFF778FFAC
:10680000F3E70025F1E7C046D064FF1FC064FF1F17
:106810007443FF1F030010B5002801D1002010BDF4
:1068200000780B4A002803D15988D1821B7913764E
:106830001378022BF2D10023984200D10333137056
:10684000044B1B78FF2B01D0FFF752FF0120E6E736
:10685000C064FF1F7443FF1F002911D000280CD013
:106860004B79012803D140225242134303E03F22D7
:106870001340032802D001204B7170474022F4E7F7
:106880000800FAE770B5094D0100287800280BD000
:10689000074C0622200005F013FA21002878FFF7A4
:1068A000DBFF200005F08CFA70BDC046E064FF1FDE
:1068B000BA64FF1F00290AD0012808D13F224B7972
:1068C0009343C02B03D0403B5A425341981C70471E
:1068D00070B5174D06002B78FF2B15D00A2005F058
:1068E00077FA041E10D0D0230370C83B8370114B7D
:1068F00011491B784670C3700622043005F0E0F998
:106900002100287804F06CFF0C4B1B78012B0DD173
:106910000B4B1B68002B03D09B68002B00D09847C3
:10692000084B04211878084A05F03AF870BDC046B3
:106930007443FF1FE064FF1FBA64FF1FDC64FF1F86
:106940000865FF1F0C65FF1F60EA0000014B986897
:106950007047C046C064FF1F014BDB681868704772
:10696000C064FF1F074B10B5DA681368013313606A
:10697000054B1878FF2803D08021C90105F0D0F815
:1069800010BDC046C064FF1F7443FF1FF7B50E0063
:1069900002F0C8F8051E1CD00E4B06621F78002FAF
:1069A00000D10778AB791020019305F011FA041E8D
:1069B0000FD0D0230380C73B8370019BE91DC370B8
:1069C0000622043005F07CF921003800E66004F06E
:1069D00007FFF7BD7243FF1F014B18787047C04691
:1069E000E064FF1F054B002805D1054B1A78054BC5
:1069F000002A00D1014B18007047C046D064FF1F29
:106A0000E064FF1FBA64FF1F014B58687047C0461F
:106A1000C064FF1F024B1868431E9841C0B2704704
:106A2000E464FF1F421E03000120152A03D9FF3B27
:106A30005A425341D8B27047F0B51C0000230E00F3
:106A400085B0039002920B70029A934201D300200A
:106A500019E0E55C5A1CD2B2002DF8D00298511909
:106A60008142F4DC0233DFB2A35C18000193FFF72C
:106A7000D9FF002807D0013D019A0399EBB233708A
:106A80008A4202D1E01905B0F0BDDB19DBB2DBE7C9
:106A900010B50C0002F09EF803001220002B03D06A
:106AA0002100588805F02CF910BD000070B50E4D7E
:106AB00084006359002B15D0186A002801D005F016
:106AC00007F92B59586A002801D005F001F92B5914
:106AD000986A002801D005F0FBF8285905F0F8F86D
:106AE00000232B5170BDC046F064FF1F1C4B70B5D6
:106AF00004000E00150099420AD11A4B1B68002BA6
:106B000001D1122070BD1B68002BFAD09847F9E71D
:106B1000154B994215D1134B1B68002B0AD01B68EB
:106B2000002B07D09847002804D1104B1C70104B45
:106B30001D70E7E729002000FFF7AAFF0028E1D138
:106B4000F3E7080001F0EEFF0028DAD00378032015
:106B5000A342D7D12900300005F0D2F8D2E7C046D1
:106B6000FEFF0000EC64FF1FFFFF0000E964FF1F51
:106B7000E864FF1FF7B50400808801F0D3FF00250B
:106B8000A84203D00578A08802F008F81C4E33789C
:106B9000002B1FD0AB421DD11A4B28001978FFF7EC
:106BA00077FF002818D000233370A3790820A77836
:106BB000A688019305F00CF9011E0DD0D0230370B7
:106BC000CA3B8370019B477086808371280004F064
:106BD00007FE01E0002DE8D1A0880B4B8200D358BE
:106BE000002B01D0FFF762FF1721A088FFF768FD97
:106BF000A08801F027FDA08801F0FEFDF7BDC0468A
:106C0000E964FF1FE864FF1FF064FF1FF0B587B061
:106C10001D000CAB1B88070001930DAB1B881420D3
:106C200002930EAB1B88160003930FAB1B880091D9
:106C3000049310AB1B88059305F0CAF8041E1AD004
:106C4000D0230370CB3B47708370C67006222900A7
:106C50000430002D11D005F033F8019B2100638131
:106C6000029B0098A381039BE381049B2382059BE5
:106C7000A37404F0B5FD07B0F0BD04F069FFECE7C4
:106C8000F7B5009308AB1B8807000C200D00160019
:106C9000019305F09DF8041E13D0280001F042FF77
:106CA00000280FD00078D0232370C93BA370009B2D
:106CB00021002381019B6770A580E680638104F039
:106CC0008FFDF7BD014B1878EDE7C0467443FF1FF9
:106CD00013B5040064890389C2888188C078009450
:106CE000FFF7CEFF13BD000010B5044C206800284C
:106CF00003D004F0EDFF0023236010BDF464FF1FF8
:106D0000A122F0B5818892004A43384B384F1B6866
:106D100004009B189D2292009B18827989B01A600A
:106D20003B68002B5FD01D78324B1B68002B04D0D2
:106D30005B68002B01D00020984726000836310000
:106D4000E079FFF7B7FD237DE0710200E07804935E
:106D5000638A29000393238A0293E3890193A3881A
:106D600000933300FFF752FFE378002B0BD1E28949
:106D7000A379A18802920196E2792800009201226B
:106D800001F0DAFEE0703B68002B20D0FFF7ACFF8B
:106D9000194D287800281AD0184B1978FFF778FE7B
:106DA000002814D02B78E67808200793A78805F0F0
:106DB0000FF8011E09D0D0230370CA3B46708370C0
:106DC00087808671079804F00BFD00232B70172134
:106DD000A088FFF775FCA08801F034FCA08801F0C2
:106DE0000BFD09B0F0BD064B9DE7C0463409FF1FFF
:106DF000F464FF1F0865FF1FE964FF1FE864FF1FBD
:106E00007443FF1FF8B5070008000E0001F08AFE6A
:106E1000041E18D02620FFF78DFC051E00D1257812
:106E2000062004F0D5FF041E0DD00021062204F038
:106E30008FFED0232370C23B21006770A370A68011
:106E4000E8B204F0CDFCF8BDF0B585B001930AAB13
:106E50001B78070002930BAB1B7808000D00009213
:106E6000039301F05FFE061E22D0102004F0B0FF55
:106E7000041E1DD01022002104F06AFE2620FFF718
:106E800059FC002800D13078D0232370C13BA37077
:106E9000009B21002372019B67706372029BA58097
:106EA000A372039BC0B2E3720C9BE36004F098FCF6
:106EB00005B0F0BDF7B50D00019001F033FE071EDF
:106EC00020D00E2004F084FF041E1BD02620FFF7E4
:106ED00031FC061E00D13E78D0232380C53B06221C
:106EE000A370F91DE01C04F0EBFE019B2A006381F6
:106EF0000123DD401A401D40210022736573F0B26A
:106F000004F06EFCF7BD0000F0B585B002901000F3
:106F10000D0017000A9E039301F004FE041E31D0F9
:106F2000029B002B2ED1039B02795B0724D51223F1
:106F300013430422002E08D10B99002905D10C9986
:106F4000002902D10D9900291AD01A430D9B2271F4
:106F5000002B00D0C9E0002E00D1CFE0002D00D0E2
:106F6000CCE0606A002801D004F0B2FE1C213000A1
:106F700004F0B6FC606205E002239A430E33D7E7C3
:106F800093432371654BBA00D458002C00D1AAE07A
:106F9000002E10D0236A002B03D11C2004F018FE11
:106FA00020625E4BBA00D358186A002803D01C2216
:106FB000310004F085FE0C9B002B12D0574CBB0017
:106FC0001D596B6A002B03D1162004F001FE686284
:106FD000BB00E358586A002803D016220C9904F02D
:106FE0006FFE0D9B002B11D04C4DBC006659B36A4F
:106FF000002B03D1142004F0EBFDB0622B59986AEA
:10700000002803D014220D9904F05AFE380001F034
:1070100089FD051E67D0414BBA00D358002B62D0C2
:107020001A6A3420002A00D11C389A6A002A01D03A
:10703000143080B20B9A002A01D01C3080B25B6AF7
:10704000002B01D0163080B204F0C2FE041E4AD0DC
:107050001822002104F07CFD2620FFF76BFB019035
:10706000002801D12B780193D0232370029B2000AC
:1070700063700A23294EA370039BBD00A371AB5913
:10708000A780196A1830002905D01C22A06004F0DE
:1070900017FE200034307359996A002907D0030085
:1070A00014221433E060029304F00AFE02980B9B52
:1070B000002B08D003001C221C330B992061029383
:1070C00004F0FEFD02987359596A002903D0162274
:1070D000606104F0F5FD6B462100187904F080FB37
:1070E0003800FFF7E3FC05B0F0BD10220D9B0D99B1
:1070F0001B69A018236204F0E3FD2CE70B9B002B17
:1071000000D13FE7012D00D03CE7606A002801D0A4
:1071100004F0DEFD1C210B982AE7C046F064FF1F37
:1071200010B5044C2068002803D004F0D1FD0023E2
:10713000236010BDE464FF1F0B4B07B51A68002ADB
:1071400001D100200EBD6946531C01201278073181
:10715000FFF772FC0028F4D00278012310001840D9
:107160001A42EED0EEE7C0460065FF1FF0B51F4F94
:1071700001203B6887B0002B25D09B78059300F059
:10718000B3FB002821D00A20FFF7D4FA04000B201B
:10719000FFF7D0FA164B05001E78731E9E413B6820
:1071A000F6B2191DD878FFF757FB3B682900DA7A49
:1071B000043303929A7901930292009033002000E5
:1071C000059A04F02DFC07B0F0BDFFF7B5FF0028CD
:1071D00005D00620FFF7AEFA04000720D8E7082004
:1071E000FFF7A8FA04000920D2E7C046E464FF1FB5
:1071F000E064FF1F70B50A4E040033780D00FF2BCA
:107200000DD0042004F0E4FD011E08D0D02303704B
:10721000CE3B45708370C470307804F0E1FA70BDE5
:107220008443FF1F70B5040006200D0004F0D0FD5C
:10723000011E0AD0D0230370CD3B8370054B4470F0
:107240001B688580187804F0CBFA002C01D0FFF77A
:1072500067FF70BDE464FF1FF8B5264F06003B686A
:107260000D001124002B05D10522234B1B7813425E
:1072700002D112242000F8BD204A10241268002AEE
:10728000F8D01278002AF5D0DB0719D52B789A1E92
:10729000012A1AD80C2004F09BFC13243860002823
:1072A000E8D000230A22437029000670023004F05F
:1072B00007FDFFF75BFF041E0AD0FFF731FFD9E798
:1072C00000F012FB0028E1D1E4E7002BE2D0D0E788
:1072D0000B4B1B78032BCDD11D20FFF72BFA094B4D
:1072E00018800028C6D0084B04211878074A04F0FB
:1072F00057FBBFE7E464FF1FE164FF1F0065FF1F4A
:10730000E064FF1FDE64FF1F0C65FF1F60EA0000E2
:10731000F7B50193194B14001A78052306000F00E6
:1073200012201A4221D0012920D1154B1D68002DB1
:107330001BD002201F2C18D8002C02D0019B002B40
:1073400013D0104B1F221E706E1C0021300004F061
:10735000FFFB01992200300004F0B2FC3100200054
:107360002C70002F06D004F0BBFCFEBD064B122093
:107370001D68DCE704F094FAF7E7C046E164FF1FFC
:107380000065FF1F8443FF1FFC64FF1FF8B50F4E0D
:1073900012243368002B17D01B780F3C834213D183
:1073A00000250B4F0221387804F04AFB094B0421D9
:1073B00038781D8004F044FB074B28001D8033689B
:1073C0005C7004F00DFB04002000F8BDE464FF1FB6
:1073D0000C65FF1FF864FF1FDE64FF1F70B50128F6
:1073E00023D11B4C2388002B03D01A4A1578002D7B
:1073F00007D0194B1B68002B02D01878FFF7C6FF87
:1074000070BD3B2B02D93C3B2380F9E7134E022190
:10741000307804F015FBFA222388920002215A43A7
:10742000307804F025FA2580EAE70B4B1B68002B27
:10743000E6D00B4B1B785B07E2D5084B022118788E
:1074400004F0FEFA0022024B1A80FFF769FED7E72C
:10745000F864FF1FDC64FF1FE464FF1F0C65FF1F5F
:10746000E164FF1FF8B51E4D2868002803D004F022
:107470002FFC00232B601B4E3068002803D004F043
:1074800027FC00233360184F05243B781800204068
:10749000234221D0154800F02BFA3B78234213D029
:1074A000202004F095FB2860002813D02022002122
:1074B00004F04EFB202004F08BFB041E306005D04E
:1074C0002022002104F044FB002004E0286804F09E
:1074D000FFFB2C601320F8BD00F00AFAF4E7C04669
:1074E0000065FF1FFC64FF1FE164FF1F7843FF1F5F
:1074F00010B50A4C23681A1E0ED0002808D101309E
:10750000587004F06DFA002805D02368002B02D0D3
:107510000021FFF787FE0122100010BDE464FF1F69
:10752000F7B5274E050033680191181E21D05C780D
:10753000244F012C30D1FFF7FFFD002825D020007B
:10754000FFF7F8F80400412814D91F4B02211878DE
:107550001E4A04F025FA1E4B3C3C1C800222336874
:107560005A703B78002B14D128000199FFF75AFE7E
:107570000120FEBDFA2292004243002AEED0124BB7
:107580000221187804F074F9E8E7FFF7D3F8020055
:10759000F3E700233B70EBE73B78002BE8D10320B7
:1075A00004F016FC011E08D0D0230370CC3B4570BC
:1075B00083703368187804F013F9FFF7B1FDD7E74B
:1075C000E464FF1FDC64FF1F0C65FF1F60EA00001E
:1075D000F864FF1F10B51749838802008B4220D042
:1075E00011D815498B4217D0144900205B1899B265
:1075F000012907D8926811785A425341D8B2FFF74F
:10760000F9FD012010BD0E4A00209B1807229BB2F5
:107610009A424041C0B2F5E783681878FFF768FFE7
:10762000F0E7836899785A78090218781143FFF7D0
:1076300077FFE7E70A20000006200000F8DFFFFFE1
:10764000AFDFFFFF014B18707047C0468543FF1F37
:1076500010B5064C207001F041FA207804F088F94A
:107660000521207800F062FD10BDC0460C65FF1FAB
:107670000BB273B50D00002B00DBC4E0884B18780B
:1076800004F01EFA041E0ED00378912B0FD0A22B0B
:1076900000D1A1E0834B1878FF2852D0210004F0DC
:1076A0009FF800284DD180200002684076BD4378C5
:1076B0000F2B76D013D8052B70D00E2BEAD18088F3
:1076C000794B98422BD8794B98421BD8784B9842EB
:1076D000E0D1A3681878591CFFF774F838E03E2B06
:1076E000D8D18378032B74D06CD8012B6ED0022BA9
:1076F000D0D1704B1B68002B23D05B68002B20D0AF
:1077000098471EE06C4BC0180C28C3D804F0A0FAB0
:107710001DC2C2150BC20B0B0B3223C23C00674BC0
:10772000C0180728B6D8664B1B68002B09D01B6809
:10773000002B06D0200098470AE0A3681878FFF7CE
:10774000C7F8200004F054F8ADE7A068FFF762F82E
:1077500000289FD0F5E7A3681B78002BF1D0554B8C
:107760001B68002BEDD01B68002BEAD02100554888
:107770009847EDE74F4B1B68002BE2D01B68002BAE
:10778000DFD021005048F3E7504B1B68002BD8D0C6
:107790005B68002BD5D021004348E9E7FFF7EAF901
:1077A000CFE780884A4B984203D04A4B984200D09A
:1077B00070E7464B1B68002BC3D05B68002BC0D022
:1077C0002100D5E7153B012BBBD963E7FFF798FAFA
:1077D000B7E7FFF77DFAB4E73F4B1B78042B07D1DF
:1077E00000236A4613800179408800F0C5FCA8E7B1
:1077F000364B1B68002BA4D05B68002BA1D0010086
:10780000364898479DE7012421420AD0294B1B683E
:10781000002B04D05B68002B01D00020984701208A
:1078200043E78B070AD5264B1B68002B04D05B6807
:10783000002B01D020009847022036E704212800C1
:1078400008400D4200D131E7254E3388002B21D06E
:10785000013B9BB23380002B1AD1FFF7DBF80028E5
:107860000AD0204B1C70164B1B68002B04D05B68A1
:10787000002B01D020009847FFF7C6F8694601F0B9
:1078800001FD6846FEF7FEFF1D20FEF753FF308026
:1078900004200AE7024B187804F0D2F8F8E7C04653
:1078A0000C65FF1F8543FF1F0E2000000120000014
:1078B000091000000465FF1FFEDFFFFFAFDFFFFFC1
:1078C0000865FF1F0C2000000B200000EC64FF1F68
:1078D0000D20000013200000E164FF1FFFFF0000E7
:1078E000DE64FF1FDC64FF1F10B501F09BF910BDC3
:1078F000014B18607047C0460865FF1F0B880020C9
:10790000162B01D817230420014A13807047C04664
:10791000B664FF1F00207047074A030011888142A8
:1079200007D091880020994202D1013080001018C0
:1079300070470020FAE7C0461465FF1FF0B58F7846
:1079400006000D00C5B01E2F15D1FFF7E5FF051E7F
:1079500003D10024200045B0F0BD00223B003100DF
:10796000C078009200F0B2FB0400A81C00F0D2FB2B
:10797000FF23EB70EEE7264B062403931B78FF2BC7
:10798000E8D0182FE6D87B08224A013BDB000292A0
:107990009A589446002ADDD0029AD3185B68002BCF
:1079A000D8D00878002802D14B78012B02D10624C8
:1079B000122FCFD107AFAB88697800976446AA68C9
:1079C000A047041EC6D1AB78029A5B08013BDB00DE
:1079D000D318390030005B689847041E0BD1AB7890
:1079E000042BB6D0039A310010782200009700F0E3
:1079F0006DFB0400AEE76A78002AABD1AA7805A92E
:107A00003B88087130000A704B80FEF747FBA0E707
:107A10008843FF1FF8BF00111D4B37B50500984282
:107A20000BD000290AD1FFF777FF002805D11948AC
:107A3000FFF772FF002800D0058037BD01291AD159
:107A4000FFF76AFF041EF8D001235B420380A3788E
:107A5000FF2BF2D0FE2B07D00023E07814220093F6
:107A600029001E3300F032FBA01C00F053FB012361
:107A70005B426380E1E70229DFD1013901F0BEF802
:107A80000028DAD12800FFF747FF041EDFD1D4E732
:107A9000FEFF0000FFFF0000022210B5074B52421C
:107AA0001A80074801325A809A80DA8000F07EFA04
:107AB000044801F025F8002010BDC0461465FF1FE2
:107AC0003D790011197A00110388F7B50400002BE5
:107AD00002D102252800FEBD426802211378254804
:107AE0005268FEF7A5FD00282ED0234F01253A88C5
:107AF000002AEFD0802321885B0201259B1A99423E
:107B0000E8DC0C2004F064F8061E31D03B882288A3
:107B10009C4600231800019561469DB2491989B21F
:107B2000AA421BD8002801D062443A8000233000CA
:107B3000082208C0210004F0C3F8104A1368002B83
:107B400013D100251660C5E76268022113780C483E
:107B50005268FEF76DFD0028C7D1BAE760681D01C5
:107B60004019418101330198D6E71A001B68E6E706
:107B70001325AFE766C000118643FF1F1065FF1F86
:107B800064C00011014B18707047C0468843FF1F46
:107B900014230A0010B51A40194204D00122102102
:107BA00001F048F810BD4B06F9D40120884340008D
:107BB000F8E710B514008B0604D50122102101F05E
:107BC00039F810BD08230A001A40194202D14BB2FD
:107BD000002B0FDA102101F02DF8002808D0230027
:107BE000F2331B78002BECD0F1342378012BE8D151
:107BF0000020E6E703208907FAD4E2E7F0B51F008A
:107C0000184B85B01C68019002910392002C27D17B
:107C1000200005B0F0BDA5683301ED186B89019A0D
:107C2000934211D3029A93420ED8002F04D10A9B9B
:107C3000002B10D12C00EBE73B002978039A6868F1
:107C4000FEF7F6FC0028F2D10136B6B2A388B342A3
:107C5000E1D82468DAE7A3680A9A5B891380E9E728
:107C60000026F3E71065FF1F37B50C000A88498826
:107C70000123914217D3002A15D0651D23792A00CC
:107C800002210A48FEF7D4FC102300280BD02379E8
:107C90006188208800242A000094FFF7AFFF0A23A0
:107CA000A04200D0230018003EBDC04666C00011AF
:107CB00013B50A0008884988012388420BD8002898
:107CC00009D00024137905320094FFF797FF0A23A7
:107CD000A04200D02300180016BD13B50A00088882
:107CE0004988012388420BD8002809D00024137941
:107CF00005320094FFF782FF0A23A04200D0230040
:107D0000180016BDF0B58BB003904A8808880E00A5
:107D10000123824255D3002853D00023012704AC0D
:107D200023700022718813000092FFF767FF051E81
:107D30003ED02078002835D12B78022B18D16770DF
:107D40006A8983000130E31880005A806968022242
:107D5000201803F0B5FF23780133DBB22370042B26
:107D600019D93B006889013080B2002BD9D01FE0BF
:107D700002236370122358436A89231804305A80FF
:107D800069681022201803F09BFF23780133DBB2CF
:107D90002370002BE5D10C4A6B899B185A42534142
:107DA000DBB2DFE76378012BE4D12B78022BC7D05D
:107DB00022780A23002A04D021000398FEF798F9BC
:107DC000002318000BB0F0BD0100FFFF0F4BF0B512
:107DD00004001868002816D083685D89A54207D87A
:107DE0008288AE18B44203DA12019A18934201D184
:107DF0000068EFE71E005F891036A74204D1002912
:107E000000D00D801800F0BD3300EFE71065FF1FB4
:107E100070B505000C0008880021FFF7D7FF0300AC
:107E20000120002B04D022002800197AFFF7C1FEA0
:107E300070BDF7B50C00002501902300EE331B78D0
:107E4000AB4201D800200AE06B00E65A0021300066
:107E5000E718FFF7BBFF002802D126800130FEBDE6
:107E6000017A0198FFF794FE002802D03B88238016
:107E7000F5E70135EDB2E0E710B504000888002110
:107E8000FFF7A4FF03000120002B03D02000197A84
:107E9000FFF77EFE10BD0000054B1B68002B01D1D3
:107EA000180004E09A6852898242F6D19888704797
:107EB0001065FF1FF0B50E27002687B0039302ABB5
:107EC000FF183E8005001F4B40891400984207D0E0
:107ED0002B78013000976A6880B2FFF78FFE0600AA
:107EE00002212B7818486A68FEF7A2FB00280FD001
:107EF0006C892000FFF7D0FF002802D0013C041954
:107F0000A4B2039B002B00D01C80300007B0F0BD52
:107F100002212B780D486A68FEF78AFB0028E7D11A
:107F200002212B780A486A68FEF782FB002807D0F6
:107F3000002EDED03B88A342DBD17489013CDFE711
:107F40006C89DEE7FFFF000066C0001164C000110D
:107F500062C0001110B50C00FFF7DEFC0300022028
:107F6000002B0AD0002C00D023609B781720FE2B1A
:107F700003D00138FF2B00D1002010BD73B50D00D8
:107F800001A904001600FFF7E5FF172805D0002E11
:107F900004D129002000FEF727F976BD0122102127
:107FA000200000F047FE0028F3D0F6E7014B1860F0
:107FB0007047C0462065FF1F37B56B469D1D010009
:107FC00004000222280003F013FF2B88B02B0ED1EF
:107FD0002379122B09D12300FA331B78012B06D108
:107FE0000121608800F0E0F801E01B2BF8D037BDDC
:107FF00010B5054B0421187000F098F8FFF74CFD00
:10800000FEF770FB10BDC0462465FF1F0020F0B5D1
:108010000BB20F0087B0834234DA274B187803F095
:108020004FFD051E2BD00378A02B25D103AE3100C8
:10803000FEF7E4F8041E0BD1B378DB0724D51F4B01
:1080400006341B68002B03D0310068889847040071
:10805000A868002801D003F04BFD002C08D1184A75
:10806000039B1340174A934206D0B3781B2B03D0CF
:108070000121688800F098F8280003F0B9FB8020FF
:108080000002784007B0F0BD0F4B1B68002B10D0EA
:10809000310068889847041EDAD07378002BD7D156
:1080A000B27801A90A704B800C716888FDF7F6FF61
:1080B000CEE70624F1E7C0462465FF1F1C65FF1FBD
:1080C00000FFFF00000112002065FF1FF7B50190BF
:1080D000FC200D0017001E0003F07AFE04001320A0
:1080E000002C12D0B02320002370089BF42267706C
:1080F000658026710830002B08D0190003F0E0FDE0
:108100002100019803F06CFB0020FEBD089903F0EC
:108110001FFDF5E710B5041E06D00078FD2803D832
:1081200003F08EFBFF23237010BD00000A1F93B2E3
:1081300010B504000220032B05D882400020024B1A
:10814000D1529B189C7010BD4465FF1F0B8870B501
:10815000043B04000D000220032B0BD8012120005A
:1081600000F04CFD03001420002B03D02900200058
:1081700000F0DEFB70BD000007B51300034A00925B
:108180000A00012100F02CFC0EBDC046B583001191
:1081900007B5019203220092024B0A00122100F05F
:1081A00049FC0EBD3384001107B56B4601AA11804E
:1081B0000449D88008780633012802D1190003F059
:1081C000CFFB07BD2565FF1F0C4B10B518700023B2
:1081D000FF210B4A1380138193819380094A5380B6
:1081E0001370517293819372D174D3821375517746
:1081F00003F09EFD00F0FCF910BDC0465465FF1F62
:108200004465FF1F2665FF1FF0B58DB06B4600204B
:1082100003910C229B5E834200DBB0E05D4B18783B
:1082200003F04EFC051E00D1A4E00378902B00D093
:108230009DE006AF01004688380000F013FA796827
:108240000400002900D19CE03B88052B6ED13B89BE
:10825000032B1CD905AC200000F0A2F86288172A75
:1082600061D83989131D994231D179682378043155
:108270000291D90738D5607800F08EF9071E06D034
:10828000002303712378012B08D0132B23D0A86877
:10829000002800D178E003F02BFC75E06288029999
:1082A00009A800F0A6F80290380000F08BF909AA9E
:1082B0002378387A0192002231000092029A00F06D
:1082C00012F9380000F064F9029B002BDFD0300077
:1082D00000F080F9DBE70378032BD8D1628802999C
:1082E00009A800F0D6F8DEE7122B13D1029909A8ED
:1082F00000F0B5F8021EEAD127498B88002BC6D0C2
:10830000887909A92378019161780091310000F002
:10831000EAF8BCE7002302AA93833000617809AA37
:10832000FFF72AFFB3E71D4B0993F6E7042B02D0B2
:108330009A1F012AABD8184A043B9B00995A00297E
:10834000A5D0D218907831003A0000F0AEF800289D
:108350009DD13B88042B03D001213000FFF724FF7F
:10836000012C04D1A868002801D003F0C1FB28002B
:1083700003F03EFA8020039B0002434018000DB03A
:10838000F0BD012800D182E701213000FFF70CFF8A
:10839000EDE7C0465465FF1F4465FF1F010017004D
:1083A0000B7803704B784370CB788A781B021343A9
:1083B000438070470A88030002700A88120A4270DC
:1083C0000A88012A06D14A8882704A88120AC27035
:1083D0000420704702208242FBD14A8804309A7000
:1083E0004A88120ADA708A881A718A88120A5A71BF
:1083F000EFE710B50400012082420CD94B780A78CF
:108400001B0213432380834206D1CB788A781B0258
:1084100013436380002010BD022BFBD1CB788A78F8
:108420001B02134363804B790A791B021343A38019
:10843000F0E70B8803700B881B0A43704B8883702E
:108440004B881B0AC3708B8803718B881B0A43718E
:10845000CB888371CB881B0AC37108207047030047
:108460000120082A14D14A780878120202431A809F
:10847000CA788878120202435A804A79087912022F
:1084800002439A80CA798879120202430020DA8076
:10849000704710B504000120022A05D100204B7856
:1084A0000A781B021343238010BDF8B50600102084
:1084B0000F00150003F08CFC04000120002C0ED0EE
:1084C000A0230C22290023806780201D002D07D0C7
:1084D00003F0F6FB2100300003F082F90020F8BD24
:1084E00003F036FBF6E7F7B51E00009008AB14204A
:1084F00017001D78019103F06BFC041E12D0A2231B
:108500000370019B47704380099B057146710C22E3
:108510000830002B07D0190003F0D2FB210000988F
:1085200003F05EF9F7BD099903F012FBF6E737B5E2
:10853000041E0FD04388002B0CD00025C1881323C4
:10854000007A172201950095FFF7CDFFFF23658084
:108550006372257037BD000010B50C4904004A88CD
:10856000002A09D08B89002B05D00020CB8A02225B
:10857000834201D010BD012213000A204343002092
:108580004032C854C81842800472F3E72665FF1FC2
:108590000023438003707047094B00211A0010B577
:1085A0005C88002C06D01C79844203D10A234B43FB
:1085B000D01810BD01310A330329F1D10020F8E7AA
:1085C0002665FF1F10B50400407A03F039F9FF2338
:1085D000637210BD7047043010B580B203F028FB01
:1085E000002803D00421494203F0CAFA10BD00005C
:1085F00070B50025104CA0682580A581A580A842F3
:1086000002D003F075FAA56000250C4C0C4B606D90
:108610001D80230058331D70A84202D003F068FA71
:10862000656500256068002801D003F061FA013516
:1086300008340A2DF6D170BDEC65FF1F9065FF1F51
:10864000E065FF1F70B5041E09D1054D2880A88183
:10865000A880A868002802D003F04AFAAC6070BD78
:10866000EC65FF1FF0B54B8885B001930023436094
:108670000A7905000F00022A00D07BE0CA88032A8D
:1086800017D98B685E7819783602DC78D8790E4372
:1086900099781B7A24021B020C43034353495BBAAB
:1086A0000B80331D93421ED1042C04D0631F022B78
:1086B0000ED9012015E0019A4D4B1201D35A002B1F
:1086C00006D00198FFF7BEFF4A4A136901331361D0
:1086D0000421B8682E812C80494203F051FA686069
:1086E000002005B0F0BD434D042C06D0631F022BC3
:1086F0000FD9EB680133EB60DBE7019A3C4B1201C9
:10870000D35A002B05D00198FFF79CFF2B6901334A
:108710002B61374B30000293019B029A1B0101939E
:10872000002301998C468B52130063449C80039371
:108730009E81FFF750FF039B041E986016D0042112
:10874000B868494203F01CFAFA880100043A200094
:1087500003F0B6FA0199029AFB888A5A043B9B18E7
:10876000029A8B522B6801332B60A2E7AB6901336D
:10877000AB619EE71E4B0293019B1E01029BF35AC5
:10878000002B2DD002998C19A068002828D0012A2E
:1087900026D1FA889B189BB27352A189994217D3AC
:1087A0009B1AC018B96803F08BFA029BA289F35A8E
:1087B000934200D07DE700222B81A3882B80A36801
:1087C0006B60029BF2520B4A53680133536070E7AF
:1087D000084A9368013393600198FFF733FF68E715
:1087E000044A536901335361F6E7C0465665FF1FDB
:1087F000EC65FF1F5C65FF1F70B5051E15D10B4CA6
:108800000B4B1880230058331870606D002802D07D
:1088100003F06EF96565250050356068002801D0C9
:1088200003F066F90834AC42F7D170BD9065FF1FC4
:10883000E065FF1FF0B51700A12285B092000193FB
:108840004243394B06001B680C009B18D933FF3399
:108850001D78FDF741FF0430854204DD3000FDF74F
:108860003BFF0430C5B2BD4207D33A0000213000BF
:10887000019B03F0CDF805B0F0BD2900380003F0EE
:108880007FFA2300C6B250331E700393019B290068
:108890006365380003F094F9CBB20293002B02D049
:1088A000039B01361E7000262300503303931B7870
:1088B000B34204D8606D002831D10020DBE7029A72
:1088C0002800002A04D0013B1000B34200D0280049
:1088D000F700E719387003F00BFA786000280ED023
:1088E0003A78019903F0ECF9019A3B780136D318F4
:1088F0000E4A0193D369F6B20133D361D4E7039BE7
:1089000018706065A74205D1084A1320D36A013365
:10891000D362B0E7606803F0EBF80834F2E703F0E5
:10892000E7F800236365C8E73409FF1F5C65FF1F94
:10893000F7B50D0007000421686803F021F92B89C1
:10894000040003702B891B0A43702B8883702B88CB
:108950001B0AC3702E8902250436F6B2F42E15D8F0
:108960001B4B9F4214D10C2003F032FA1135011E2B
:108970000CD0902303708E3B0371043B4380154B56
:108980008460C680187802F02BFF00252800FEBD09
:108990005C237B43104AD3180093583301931B7810
:1089A000002B0FD10300320038000099FFF742FF7F
:1089B000019B05001B78002BE8D13800009902F0DC
:1089C000B7FFE3E7054A0725536A01335362DDE742
:1089D000FEFF00005465FF1F9065FF1F5C65FF1FD1
:1089E000F0B587B0009017200F0016000193FFF735
:1089F000F2FD1325041E19D00C98031E02D0019914
:108A0000201D9847030AE370052302AAA0700430D2
:108A1000908127700098667003A993800494FFF7F3
:108A200087FF051E02D0200003F062F8280007B07F
:108A3000F0BD0000F0B587B01F000CAB1B780391B0
:108A4000059301210DAB06001C78049200F0D6F8C6
:108A50001425002821D02000FFF77EFD0135041EDB
:108A60001BD01149059B0A7803700132D2B2131E44
:108A7000C68001D101231A000B7022713000049BC3
:108A800003990097FFF7ACFF051E09D123002100D1
:108A90000648074A093303F0E3F8280007B0F0BDA1
:108AA000002363802370F8E75865FF1F2F850011AE
:108AB00030750000F8B505000E00064C064F23681F
:108AC000002B02D03100280098470434BC42F6D174
:108AD000F8BDC046FC65FF1F1066FF1F0123064A54
:108AE0005B425380002313715362044A1360536046
:108AF0009360D360136170471066FF1FFC65FF1F12
:108B00000200002310B506499C000859002801D135
:108B1000625010BD0133052BF6D11320F9E7C04692
:108B2000FC65FF1F034A5388181A434258414042CC
:108B3000104070471066FF1FF0B585B002930AAB76
:108B40001F780CAB1B88009008000E000192039365
:108B5000FFF7E8FF05001120002D1BD10E48FFF79D
:108B6000E1FF04001520002C14D006220B99A771F8
:108B7000E01D03F0A5F8019B30002371029B290042
:108B80006371009B66802370039B6562E381FFF73E
:108B900091FF280005B0F0BDFFFF000010B5FFF702
:108BA000C1FF04000220002C12D060880121FFF7D1
:108BB00081FF606A002801D003F08AF82822002192
:108BC000200002F0C5FF012300205B42638020717A
:108BD00010BD000030B5074A074C558801001378D6
:108BE0000020A54204D05B1A59424B415842104024
:108BF00030BDC0461066FF1FFFFF0000084A10B5D9
:108C000001230C00904208D0FFF78CFF031E04D014
:108C1000037923405A1E9341DBB2180010BDC046B1
:108C2000FEFF0000024B1879431E9841C0B2704706
:108C30001066FF1F70B504000D001600FFF772FFED
:108C4000002804D10D4B9C4200D0143070BD416A05
:108C500003790520002907D012221A40102A02D1D8
:108C60000520002EF2D10F20DB06EFD5897E0C20E7
:108C7000A9428941494249420840E7E7FEFF000016
:108C8000030010B5002800D110BD0348034A4188F5
:108C90009142F9D09847F7E71066FF1FFFFF0000E9
:108CA000002330B5C45CCD5C6C40D4540133102B30
:108CB000F8D130BD0F23002210B5C45C64002243FC
:108CC000CA54C25CD209013BF7D210BD02000100B8
:108CD00010B52032103103F033F810BDF0B58BB071
:108CE0000390102005931700049102F071FF00908B
:108CF000102002F06DFF009B13240190002B05D083
:108D000000280CD11324009802F0E2FF019B002BF5
:108D100002D0180002F0DCFF20000BB0F0BD1020E4
:108D200002F056FF0600102002F052FF1324050047
:108D3000002E00D1AEE0002819D01022002102F050
:108D400007FF32002900039802F0FAFF041E0ED13B
:108D500033787F2B51D830000099FFF7ABFF009B91
:108D60001B787F2B53D801990098FFF7A3FF3000A1
:108D700002F0AEFF002D02D0280002F0A9FF002C67
:108D8000C1D1102002F024FF0600102002F020FFC5
:108D90000290002E7CD0002878D03A000F322300B9
:108DA0000125121105D00F333B4015B25A425341F1
:108DB0001BB26A1E1201002B33D0049BD2B298184A
:108DC0000099029AFFF76CFF013D1022002130004C
:108DD00002F0BEFEADB2049F2D017D19AF4242D01C
:108DE000002C33D0300002F073FF029B002B00D127
:108DF00089E7180002F06CFF85E729003000FFF7D3
:108E000059FF28002549009AFFF74AFFA7E72900E4
:108E10000098FFF74FFF28002049019AFFF740FF15
:108E2000A5E70F210F4004998A18D9B28F4208D9BB
:108E3000D15C06A819540133102BF6D1029A01997E
:108E4000C0E7791A48424141C901F2E739003000D0
:108E500006AAFFF725FF3200039806A902F070FF6B
:108E600010370400BAE7002CBCD13000029906AAE2
:108E7000FFF716FF320006A9039802F061FF0822EF
:108E800004003100059802F01BFFABE71324A9E7AB
:108E90001324AAE7002800D06EE733E76CC0001166
:108EA000F0B58BB00F0016000225009000283FD0CF
:108EB000002A3DD00B1DDBB21800029302F088FEA1
:108EC0001135041E34D0FDF747FD05003A00009926
:108ED000201D02F0D5FCEBB20393E3702B0CDBB248
:108EE0002F0A00936370FFB22B0E2370A7700193BB
:108EF000FDF72CFD1022010006A802F0C1FC2100A4
:108F0000029A04AB06A8FFF7E9FE051E0DD1039BEC
:108F100008223370009B04A9B370019B7770F37033
:108F2000301D02F0ADFCFDF71DFD200002F0D0FE6B
:108F300028000BB0F0BDF0B58FB00D00149E03906B
:108F400004920593002A03D1022420000FB0F0BD43
:108F5000002EF9D00398FFF7E5FD1424071EF4D086
:108F60007278337812021A43B3781B041343F278F1
:108F700012061A43036A0192934201D30133E3D1EB
:108F8000002D03D03B7901249B07DED50822002168
:108F900006A802F0DDFD059B13240433DBB21800A4
:108FA000029302F015FE051ECFD0059A04990430F5
:108FB00002F066FC04223100280002F061FC390056
:108FC000102210310AA802F05BFC2900029A06ABBD
:108FD0000AA8FFF783FE041E0FD1082206A908A8DD
:108FE00002F04EFC0822311D08A802F0D9FD01282C
:108FF00007D101990398FDF7C9FC280002F068FE2B
:10900000A3E70124F9E7000070B51C4C05002368B4
:10901000181E10D0002D14D11A78002A0CD1981CDB
:10902000083202F04DFE02F00BFE0135002808D197
:1090300023681D70012070BD0A331800082202F059
:109040003FFE2368002BF5D0122002F0C1FE061E61
:109050000DD0C12321680370457002311022023007
:1090600002F02EFE23683100587802F0B9FB206828
:1090700002F02EFE00232360DCE7C0463866FF1FA7
:10908000F8B504002020FDF755FB0D4EA700BB5995
:109090000500002B0DD000280BD0D878FF2809D16F
:1090A00008492A000C55F35907480333611802F0A8
:1090B000D7FDF8BD290002F02BFE0028F0D1F8E71B
:1090C0005466FF1F3C66FF1FD9A2001170B5064D04
:1090D00084006359002B05D0D87802F0B1FBFF2241
:1090E0006359DA7070BDC0465466FF1F70B5060044
:1090F0008CB00C00150000213022684602F028FDDB
:1091000031001022684602F0BBFB1D202100032223
:10911000684402F0B5FB6846FFF7D8FD2D21040036
:1091200003222800694402F0ABFB20000CB070BDA4
:10913000F0B50700160097B001931CAB1D783022E4
:109140001EAB00910AA800211C7802F001FD10223C
:1091500039000AA802F094FB1022002102A802F0B4
:10916000F7FC0722310002A802F08AFB072202ABBB
:109170009818631E9C41019902F082FB02AB9C731C
:109180002B005A1E934102AAD3730021102206A875
:1091900002F0DEFC06221D9907A802F071FB1A20DE
:1091A00002ABC01806221F9902F06AFB1022009938
:1091B0000EA802F065FB102202AB0EA908781C78FD
:1091C000013A6040D2B2087001330131002AF5D172
:1091D0000AA8FFF77BFD102212A904000EA802F0D6
:1091E0006FFD102206AB0EA908781D78013A684081
:1091F000D2B2087001330131002AF5D10AA8FFF775
:1092000065FD044310222098E4B212A902F038FB55
:10921000200017B0F0BD70B50E0014008CB0010036
:10922000102268461D0002F02BFB3100082204A822
:1092300002F026FB2100082206A802F021FB684666
:10924000FFF744FD04001022280008A902F018FBD3
:1092500020000CB070BDF8B506000D0000243719D1
:10926000AC4200D3F8BD02F06BFB030A3B70631CF9
:10927000DBB201379D4203D90234F054E4B2EEE789
:109280001C00EDE773B506000C000225002819D07C
:10929000002917D0032101A8FFF7DDFF6B469A795B
:1092A0003F231A40013313436A463000937101A9EA
:1092B0002200FFF71BFF051E04D10322E01C01A9B9
:1092C00002F0FEFC280076BD03785807DA08C00FCC
:1092D000D20080009B0710439B0F1843C0B2704719
:1092E00007230B40C908C9000B43037070470000F7
:1092F00070B50400FFF7EAFE134DA4006359002B7C
:1093000021D0186A002801D002F0E2FC2B59986E97
:10931000002801D002F0DCFC2B59D86E002801D0C7
:1093200002F0D6FC2B59186F002801D002F0D0FCB7
:109330002B59586F002801D002F0CAFC285902F0BE
:10934000C7FC00232B5170BD5466FF1F0E4B8000DD
:10935000C35870B50C00002B0FD09D68002D0CD0A9
:109360002B78201D0B706B784B70A97CFFF7B8FF32
:109370002B7E23726B69E36070BD102200212000F8
:1093800002F0E6FBF8E7C0465466FF1F014B186089
:109390007047C0465066FF1F074A0300800082588E
:1093A00010B5002A06D0D088984203D1012901D1F6
:1093B000FFF79EFF10BDC0465466FF1FF0B5264E56
:1093C00095B087000B93BB590500099112200A92B2
:1093D000002B31D0D888FFF7A5FB04001420002C07
:1093E0002AD0280010A9FFF7B1FFBB591E781D6ACB
:1093F000002E23D00895FDF7EFFA07000020FDF7B7
:10940000F1FA0790A379E61D069310AD0CA9089810
:1094100000F0E2FA0EA9280000F0D7FA0B9B0A9997
:109420000493069B09980293079B03960193009768
:109430000EAB0CAAFFF77CFE15B0F0BDFDF7CCFA21
:1094400006903000FDF7CEFAE31DA779079310AB25
:1094500006000893DAE7C0465466FF1F30B50C4C8F
:1094600085002A59030085B00120002A0ED018007B
:109470006946FFF76BFF2B591A78D888054B002AED
:1094800000D1054B6A46072100F0D9FB05B030BD7D
:109490005466FF1FCB990011D999001130B5094CC2
:1094A0008500295985B010226846253102F008FC54
:1094B0002A591121044BD0886A4600F0C0FB05B040
:1094C00030BDC0465466FF1F759A001130B5094C77
:1094D0008500295985B010226846353102F0F0FB2D
:1094E0002A591121044BD0886A4600F0A8FB05B028
:1094F00030BDC0465466FF1FB39A0011F7B54D4FFB
:1095000086001020F4590D0002F062FBF35920622E
:10951000186A132200286CD0033A29009C6802F0D4
:10952000CFFBF3591A780192002A58D11E6A227D86
:10953000317B944651400122019F114201D167467F
:109540001740217D914339432175377B4F40BC46FD
:1095500060460027800701D44F08174001210220F0
:109560008F40227D82433A432275377B5740BC4669
:1095700060460027400701D497080F400420227D51
:10958000BF0082433A432275627D002794466046BD
:10959000727B42400A4201D167460F400121627D41
:1095A0008A433A436275777B5740BC466046002742
:1095B000800701D457080F400220627D7F0082435C
:1095C00017436775767B00227E40760701D4BA0880
:1095D0000A400426617D9200B1430A4362756A78AD
:1095E000002A08D06278002A05D005220533DA77F0
:1095F00000221000FEBD04222979114205D1A17C70
:10960000114202D10533033AF1E7019A21782C780F
:10961000002A02D10A002100140018220429E8D8E7
:10962000042CE6D805206043034A05331218525C27
:10963000DDE7C0465466FF1F7CC0001110B50A006C
:109640001121024B00F0FBFA10BDC0460F9B001128
:109650000B0030B587B001AD2B806B4604001100C4
:10966000981D082202F02CFB2A000B212000024B3F
:1096700000F0E5FA07B030BD379B001110B50A00C5
:109680001121024B00F0DBFA10BDC0468B9B00118C
:1096900013B50B0011006A4613706B4604000622D6
:1096A000581C02F00DFB6A4608212000014B00F017
:1096B000C6FA13BDAB9B001110B50A001121024B75
:1096C00000F0BDFA10BDC046FB9B00117FB5050040
:1096D0000B4BAA00D4580800002C0FD0666F237FD4
:1096E000E28821780396266F0296E66E0196A46EB4
:1096F0000094FDF709FC2800FFF7FAFD7FBDC04686
:109700005466FF1F10B51721FFF7E0FF10BD0000E2
:1097100070B50A000D00064B0221040000F08FFA1C
:10972000060029782000FFF7D1FF300070BDC04649
:10973000DB9A001170B586B000236A461370836807
:1097400004001D78681E0A2859D801A902F098FA69
:10975000060633373B3F43474B4F5300180000F09A
:1097600042F9062312284BD000281BD16088FFF74E
:10977000D9F90823002813D04279002A47D1264B73
:109780001A78072312070BD5244B1A680723002ADF
:1097900006D01668002E03D0290001AAB0470300A6
:1097A0006A4613706B461B786088002B2AD1FFF73E
:1097B00067FC06B070BD180000F06CF9D4E7180023
:1097C00000F087F9D0E7180000F093F9CCE7180013
:1097D00000F0ADF9C8E7180000F0C3F9C4E71800BD
:1097E00000F0F6F9C0E7180000F0F6F9BCE7180041
:1097F00000F013FAB8E7180000F013FAB4E70723F3
:109800006A46137069466088FFF782FFD1E7052337
:10981000012AC5D1024BB8E7E164FF1F4C66FF1F68
:109820005066FF1FF8B52C4F8600F35904000D0059
:10983000002B40D0DA8882423DD15A78062A33D1B3
:109840001A78002A2ED0012099681A6A097D0142EF
:1098500006D0157B054203D007225A700120F8BDBF
:109860000220014204D0157B054201D00922F4E711
:109870000420014204D0127B024201D00B22ECE70B
:10988000164B1B68002BE9D05B68002BE6D020004C
:109890009847BB5900215B78122BDFD12000FFF7DE
:1098A00015FFDBE70E4BECE7112A04D1002900D0AD
:1098B00032252900F2E7002D08D12000FFF732F908
:1098C000002803D0102302791343037121002800DC
:1098D000FDF798FAC2E7C0465466FF1F4C66FF1FAB
:1098E0005066FF1F70B50E4E8500AB590400002B6B
:1098F00013D01B78002B11D10A4B1B68002B04D00E
:109900005B68002B01D02000984773595B78122BBD
:1099100003D100212000FFF7D9FE70BD024BECE718
:109920005466FF1F5066FF1F4C66FF1F094B8000E7
:10993000C3581020002B0CD01A6A002A09D09B684B
:10994000002B06D0127A1B7E101C9A4200D9181CDC
:10995000C0B270475466FF1F70B503000D001400BD
:109960000220002A30D000292ED013700B78081D59
:1099700053704B789370FFF7A7FCE0700120022131
:109980002B7A23716B7B034063716A7B0A4013431C
:10999000042263716E7B1640334363716E7BF6085D
:1099A000F600334363712B7B0340A371287B014096
:1099B00000200B43A371297B0A401343A3712A7B28
:1099C000D208D2001343A37170BD10B50A00010084
:1099D0000120FFF7C1FF10BD10B50A0001000220F1
:1099E000FFF7BAFF10BD70B506000C000220002E74
:1099F00030D000292ED07378201D0B70B3784B70B7
:109A0000F178FFF76DFC01223579257271794B10E1
:109A1000080013409340104003438810104080001A
:109A2000C9080343C9000B436373B1794B100800A5
:109A30001340934010400343881002409200C9082D
:109A40001343C9000B4321202373FCF773FE8542A7
:109A500001D2122070BD2220257AFCF76BFE8542D0
:109A6000F7D823781820042BF4D86378012BF1D889
:109A70000020EFE7030010B50220002909D0002BD9
:109A800007D00322481C0A7019000D3202F018F9A1
:109A9000002010BD03000222080010B5002B06D0E4
:109AA000002904D00E32591C02F00AF900221000DD
:109AB00010BD030010B50220002909D0002B07D0EB
:109AC0000422481C0A7019000C3202F0F9F8002038
:109AD00010BD10B5FFF7DEFF10BD03000220002906
:109AE00006D0002B04D0052200200A701B784B7092
:109AF000704703000220002B08D0002906D05B78B5
:109B000000200B70013B082B00D918307047030070
:109B100010B50220002909D0002B07D00622481CCE
:109B20000A7019000A3202F0CBF8002010BD10B5FF
:109B3000FFF7B0FF10BD02000B00022010B5002996
:109B40000ED0002A0CD00721197011885970118885
:109B5000090A997011180822D81C02F0B1F80020E7
:109B600010BD03000A00022010B5002B0CD0002904
:109B70000AD099785878090201431180901CD91CA9
:109B8000082202F09DF8002010BD030010B502204D
:109B9000002909D0002B07D00822481C0A701900A0
:109BA000921802F08DF8002010BD02000B00022078
:109BB00010B500290BD0002A09D00921197011789D
:109BC00018185970511C062202F07AF8002010BDB6
:109BD00010B5FFF75FFF10BD02000B00022010B5AB
:109BE000002A09D0002907D05178197011180622CF
:109BF000581C02F065F8002010BD030010B50220CB
:109C0000002909D0002B07D00A22481C0A7019002D
:109C1000063202F055F8002010BD10B5FFF73AFFEC
:109C200010BD02000B00022010B5002A06D000294A
:109C300004D018005178FFF753FB002010BDF0B599
:109C400085B017001E006A460623050008009181B2
:109C50009380FEF7C0FC1324011E02900CD0380044
:109C6000B047041E05D1280001A9FEF76FFA041EB3
:109C700002D0029801F03CFF2800FFF701FA200013
:109C800005B0F0BDF0B504008BB0019115000021C6
:109C9000102202A801F05CFF334EA700B85900283B
:109CA0003CD0C388A34239D10378002B36D1427807
:109CB000062A18D102000100553235310C3006ABAE
:109CC000FFF7A9FA002829D12000FFF72FFE020094
:109CD00006A902A801F0F4FF200002A901F070FE1D
:109CE00001200BB0F0BD816E002917D00B8A112A1C
:109CF00028D19D420ED101981231093A01F050FF4E
:109D0000012807D1BB5920009D6EFFF70FFE2900E7
:109D10000200DEE732212000FFF7D8FC2000FEF72A
:109D200001FF061E1BD0416A002918D00B8AAB42E6
:109D300015D108220198123101F032FF01280ED10D
:109D4000716A0AE09D42E9D108220198123101F0BE
:109D500027FF0128E2D1BB59996E8A7EB9E720001E
:109D600001F036FDBCE7C0465466FF1FF0B56B4DF1
:109D700087007E5985B0337802900393002B00D082
:109D800087E0B368346A01937078062817D10122FE
:109D90001B7D134202D0217B114218D102221342B3
:109DA00002D0217B114251D10422134203D0237BE4
:109DB000134200D08BE0019B5A7DEB5991E00738AC
:109DC0000428F8D801F05CFF032E42678300B36ECD
:109DD000002B03D11C2001F0FBFEB066EB599C6EFA
:109DE000002C1CD010220021200001F0B1FE0298AE
:109DF000FFF79CFD01002000FFF72DFA01F0A0FD08
:109E00002082200008211230FFF725FA0298FFF780
:109E10008DFDA076EB592100D888FFF70FFC0822B2
:109E2000EB591CE0B36E002B05D01A00198AF0889C
:109E30001232FFF70DFC0222019B197DEB591142F2
:109E40003DD0207B10423AD0073208E0F488FCF77E
:109E5000DBFD01002000FFF711FC0A22EB595A70CC
:109E6000029B9C002A595378073B042B11D8D088B9
:109E7000FEF758FE00284ED0C3895A08D218284948
:109E8000029B0298CB542B5941180433254801F00A
:109E9000E7FE05B0F0BDFCF79FFD03000120834203
:109EA00001D100200393EB59DE88FCF79BFD039959
:109EB00002003000FFF7ECFB019AEB59117D042200
:109EC00011420CD0217B114209D00B22C7E7F68842
:109ED000FCF73CFD01003000FFF7EEFB6BE7019A59
:109EE000527D01210A4204D0607B084201D00C223D
:109EF000B5E702210A4204D0607B084201D00E225D
:109F0000ADE704210A4204D0627B0A4201D010224C
:109F1000A5E71222A3E7FA225200B0E75466FF1F1A
:109F20005866FF1FE3A2001110B5064B1A780423F0
:109F3000100018401A4200D00348FFF727FA00200B
:109F400010BDC046E164FF1F8C43FF1F70B50400C5
:109F5000FFF7D4FA051E43D12000FFF77FFA234E06
:109F6000A400A0598268937CDB0708D50321036A0B
:109F70001B790B40012B02D1017F0B430377431D5B
:109F8000D97F8B1E022B0DD8022900D00121C08859
:109F9000FCF790FF042133591A7F59700A431A774E
:109FA000280070BD01290CD102231022437000212A
:109FB0000C3001F0CDFD305910213530FFF74BF951
:109FC000EEE70529ECD10223D118437010220C30A2
:109FD00001F076FE04233259117F0B431377EAE731
:109FE00008251828DCD1053DDAE7C0465466FF1F76
:109FF000F0B58BB0059143887E4F9E00F459150053
:10A000000493002C15D1012902D000200BB0F0BD23
:10A01000101D57781678FFF757F9EB683200029356
:10A020002B7A0499019300903B002000FCF70CFF71
:10A03000EBE7E388049A934201D00820E6E723780F
:10A04000012B00D1D4E0059B581E092800D9CFE090
:10A0500001F016FE05CE0A29CC506C859AB2290073
:10A060000498FFF773FFD1E7200029001022453044
:10A0700001F026FEB9594B78042B02D1013B4B70FD
:10A08000C3E70B000A00253335320C310498FFF783
:10A0900095F90498FFF702FA0522431E9841BB592F
:10A0A000C0005A70B2E7200029001022553001F09C
:10A0B00007FE049B4F4C9D00295904980A0006ABEB
:10A0C00055320C31FFF77AF929591022453106A88B
:10A0D00001F066FD012808D10498FFF7F7F9059013
:10A0E000002804D106222B595A7005988EE70823C0
:10A0F0000593FAE763780C2B7AD1E36E002B03D13A
:10A100001C2001F065FDE066BB59D86E00286FD0B9
:10A110001022290001F0D4FDBB590498DC6EFFF732
:10A1200005FC0D22A076BB595A706EE7E06E002840
:10A130005ED063780D2B5BD12B8808220382A91C8B
:10A14000123001F0BDFDBB599A68517D02221142C7
:10A1500026D0186A407B104222D00C32E4E76378A4
:10A160000E2B45D1236F002B03D1162001F030FDBB
:10A170002067BB59186F002803D01022290001F076
:10A180009FFD0F22BB59CFE763780F2B30D1206F93
:10A190000622691C103001F093FDBB599A68517D6D
:10A1A0000422114203D0196A497B1142D5D1002102
:10A1B0000498FFF78BFA28E7636F002B0DD0BB598B
:10A1C000586F0028F3D01022290001F079FD0122F8
:10A1D000BB5952425B6F1A61E9E7142001F0F8FCA9
:10A1E000BB5960675B6F002BE9D126E72978DFE771
:10A1F00007200BE75466FF1F10B5064C207001F0D6
:10A20000D7FB06212078FDF791FF0348FEF778FC85
:10A2100010BDC0466766FF1F9993001100200BB266
:10A2200070B50D00834216DA264B187801F048FC11
:10A23000041E0DD00378922B0ED0A02B37D0224BCA
:10A240001878FF283AD0210001F0CAFA002835D149
:10A2500080200002684070BD43780E2B0BD03E2B4F
:10A26000EDD18378052B12D0082BE8D18179808835
:10A27000FFF7D8FA08E0154B82889A42DFD183684D
:10A280001878591CFEF7C0FE002817D1D7E7104BED
:10A290001B785B0712D50F4B1B68002B0ED09B68F9
:10A2A000002B0BD0C289811D80889847ECE7FFF70F
:10A2B00041FAA068002801D001F01AFC200001F04A
:10A2C00097FAC5E76766FF1F8543FF1F1820000048
:10A2D000E164FF1F5066FF1F10B50078FFF712FA08
:10A2E00010BD10B50078FFF7FDFA10BD0C234343F5
:10A2F000084A10B59B185A68002A03D0012901D1D9
:10A30000904710BD9B68002BFBD00029F9D19847DE
:10A31000F7E7C0468466FF1F01238340094A10B552
:10A32000946B1C439463506B98435063D46B200030
:10A330009843012901D120001843D063116B0B43CE
:10A34000136310BD00800040F0B500240127154BB9
:10A3500085B0DA6B144E03921A6C0192DA64019B99
:10A36000E3403B4217D0039DE5403D400295E5B2F6
:10A3700002992800FFF7BAFF316A736A002908D0F2
:10A380003900002B01D0029979402800FFF7C4FF63
:10A3900001E0002BF9D101340C36172CDFD105B0C8
:10A3A000F0BDC046008000406866FF1F064B0121DB
:10A3B0005A68C2400A4204D01B68C34018000840D3
:10A3C00070471B6DF9E7C046008000400122064B34
:10A3D0008240002903D0D9680A43DA607047D968FF
:10A3E0009143D960FAE7C0460038004030B50324F5
:10A3F00044430F4BE25C1B199C785D7801232D1BB5
:10A400000135AB40013BA340A140DB430C001228C7
:10A4100007D8084992005218116819402143116069
:10A4200030BD054A11680B4023431360F8E7C0466E
:10A43000C3C0001108F0004014F00040C21F70B506
:10A44000D4B20623092C0BD80125084C95400029CD
:10A4500008D00021FFF7CAFF23682B4323600023A5
:10A46000180070BD2368AB43F8E7C04600380040D1
:10A47000214BF0B51B185B78022B21D103244443F8
:10A480001E4A1F4EA35C12199478012215008540C4
:10A49000B76B013CE4B23D43A240B563194C1228AE
:10A4A00015D89B0000290CD117495B1899680A43FD
:10A4B0009A600123205C154A834011680B431360A6
:10A4C000F0BD11495B18996891439960F1E70E4B13
:10A4D00000290DD159690A435A61225C1328E8D03A
:10A4E0000123203A93400A49086803430B60E7E7D9
:10A4F000596991435961F0E76866FF1FC3C00011B5
:10A500000080004008C1001100F00040A0F00040B1
:10A51000A4F00040F8B500241B4E1C4D1C4B1B5DE5
:10A52000012B1FD1194A9269E2401A420BD0012235
:10A53000B25693402200143AD2B2022A09D81549E1
:10A540004A6913434B61013402360C35172CE5D1AF
:10A55000F8BD0022B2560F499200521891680B4381
:10A560009360F0E7022BEED1E7B23800FFF71EFF51
:10A5700001235840C1B23800FFF77AFF3800FFF7D7
:10A5800015FF6877DFE7C04695C000116866FF1FBA
:10A590006966FF1F00F00040012202388240054B2F
:10A5A000002903D059690A435A6170475969914398
:10A5B0005961FAE700380040F8B50E0001210F009C
:10A5C0008740114A0400D368FD43BB43D360831E18
:10A5D0008B4201D8FFF7E0FF00212000FFF72EFF9C
:10A5E0000A4A0B4B5168012E05D139431B195160A2
:10A5F0005E700020F8BD2940516002221C19627073
:10A600009A6915409D61F4E70038004000800040E1
:10A610006866FF1F012210B58240074B002906D053
:10A6200019680A431A600121FFF7C6FF10BD1968B7
:10A6300091431960F7E7C046008000400C2370B5D5
:10A64000002543430A4A29009B181D70094B04004A
:10A650001B185D70FFF7B0FF0123A34006492800D7
:10A660000A681A430A6005490A689A430A6070BD7D
:10A670008466FF1F6866FF1F348000403080004002
:10A6800070B504000E00FF2813D003250540FFF726
:10A69000D5FF084AA3089B009B183F22ED00AA4063
:10A6A000AE40196820009143314319600121FFF742
:10A6B0008DFE70BD18380040F8B50C244443134B90
:10A6C0000500E4186368002B03D1A3681220002B57
:10A6D0001AD0022201270E4B00215B195A70280064
:10A6E0002770FFF769FF63681E1E08D0A3683E004D
:10A6F000002B04D02800FFF759FE4640F6B2280090
:10A700003100FFF709FE0020F8BDC0468466FF1F38
:10A710006866FF1FF7B5C420FF222B4B8000195835
:10A72000002491433F3A0A431A508022274F520295
:10A73000274E1A60274B1D5D002D21D0A31E012B33
:10A7400003D80121E0B2FFF727FF012D18D11F4BDD
:10A750009B69E3402B4213D0E3B218000193FFF74B
:10A7600025FE01000198FFF755FFE3B2143B022BD1
:10A770001DD801217156184A8D405369AB4353616E
:10A780003B7F002B0DD0E5B22800FFF795FF280096
:10A79000FFF70CFE7B7F0100834202D02800FFF709
:10A7A000A5FD01340C370236172CC3D1F7BD0121AA
:10A7B00000237156F3568D40074A9B009B189A68F8
:10A7C000AA439A60DCE7C04600E100E06866FF1F2C
:10A7D00095C000116966FF1F00F0004070B50E00C3
:10A7E00015000400FFF72AFF0C236343094A2000E9
:10A7F0009B189D605E60FFF75FFFF021064B074AE4
:10A800008900051E5A5002D02000FFF717FF2800CC
:10A8100070BDC0468466FF1F0000FF1F49A30011E2
:10A8200070B5134D07202C78002C1FD198222100E1
:10A830005200280001F064F80123C420FF222B708D
:10A840000C4B80001C635C630B4B1C605C600B4B0F
:10A85000195891433F3A0A431A50802252021A6013
:10A860000D20074A074900F0DBFF200070BDC046FD
:10A870006866FF1F00800040A0F0004000E100E09B
:10A8800015A7001115A50011030010B50620072B10
:10A8900009D8054A137000F0CBFFD7210020034BE5
:10A8A000034A89005A5010BDB443FF1F0000FF1F28
:10A8B000D11BFF1F70B51D0002240C2910D8094AB6
:10A8C000CA40D2070CD5FBF741FF041E08D1059AF8
:10A8D00004992800FBF756FFFCF7C4FDFFF724FBA3
:10A8E000200070BD1210000030B50D7802232C003E
:10A8F0009C43184201D02B431C0008252300AB4386
:10A90000284201D02B00234320241D00A5432042D0
:10A9100001D01C4325002A230D70184204D0117861
:10A920001E3B0B43137030BD0028FCD10C21137863
:10A930008B43F7E7F8B51D0006AB1B88140007AA88
:10A940000E000B201778002B27D10A78022A49D154
:10A950004A68507811780002244A08438018042875
:10A9600040D801F08DF903121D1B2300F06801F09F
:10A970001FF9021CC0B2B84200D93A1CD2B2200062
:10A98000F1682A8001F09CF906E00222F3681B8836
:10A990002A8023701B0A63700020F8BD0622EEE7B0
:10A9A00001232B80F3681B782370F5E7F368002BF5
:10A9B00016D008222A801A8822701A88120A627019
:10A9C0005A88A2705A88120AE2709A8822719A886C
:10A9D000120A6271DA88A271DB881B0AE371DBE775
:10A9E0002B80D9E701202B80D7E7C04600D6FFFF98
:10A9F000F7B516000A781D0008AB1F880C0001236C
:10AA0000022A18D14A685078117800022B4A08436C
:10AA1000801803280FD801F033F902254439E06883
:10AA200001F0C6F8C0B20723B84204D37B190193E2
:10AA3000152B02DD0D231800FEBDE0682A00310051
:10AA4000C01901F03DF96B4600209B88E268D054A4
:10AA50001B4B1B68834203D01B68834200D098477E
:10AA60000023E8E70B23002FE5D1022DE2D1737814
:10AA700032781B021343E2681380114B1B68002BD2
:10AA8000EED01B68002BEBD00120E8E70B23002F52
:10AA9000D1D1062DCED12A003100E06801F010F9A5
:10AAA000DEE70B23002FC6D1012DC3D132787533D9
:10AAB000012AC0D8E3681A70D2E7C04600D6FFFF6B
:10AAC0007468FF1F70B50C001500072837D801F017
:10AAD000D7F8041436361B36242E182015290BD827
:10AAE000184E16220021300001F032F82200290011
:10AAF000300001F0E5F8002070BD18200229FBD1DC
:10AB00001288114B1A80F6E718200829F4D10A00A0
:10AB10000E48290001F06CF9EDE718200129EBD16E
:10AB20000B4B10780B49DA69FFF7DEFEE3E71820DC
:10AB30000129E1D1064B10780749DA6BF4E70220CE
:10AB4000DAE7C0465C68FF1F3244FF1F2844FF1F3E
:10AB5000B843FF1FE043FF1F0044FF1F030010B571
:10AB60000020DB0704D50721024A034800F08CF8D7
:10AB700010BDC04620C10011B843FF1F054A0300A5
:10AB80001068002803D082889A4201D180687047FB
:10AB90000068F6E76C6AFF1F0A88030008009A4203
:10ABA00004D08A8804309A4200D000207047000008
:10ABB000F8B5F22200230D4F0D4E7968050042438F
:10ABC0003370994200D07B600A4C0021200000F0D5
:10ABD000BFFF00231A007C60AB4202D1002033701B
:10ABE000F8BD01332280DBB2F234F5E7646BFF1F5E
:10ABF000626BFF1F706AFF1F73B56B460190060002
:10AC0000684615001980FCF75FFF041E11D1002D66
:10AC10000FD07689002E11D00C2000F0D9FF00282B
:10AC20000ED0084A0460136886808560002B02D12C
:10AC30001060200076BD1A001B68F7E70224F8E7D1
:10AC40001324F6E76C6AFF1F012100220A4B10B59E
:10AC500049420A4C198099809A719A70084B207069
:10AC6000012019805A60FFF7A3FF2078FCF78AFFC4
:10AC70000448FDF745FF10BD7C68FF1F6C6BFF1F8C
:10AC8000646BFF1F35AD0011022310B5002802D000
:10AC9000FFF7B2FF0300180010BD0000030010B55D
:10ACA0000020DB0704D50421024A0348FFF7A4FF74
:10ACB00010BDC04634C100113844FF1FF0B50E2648
:10ACC00087B003930CAB1F8802ABF6180500080091
:10ACD00031000292FDF77AF804000120002C0FD019
:10ACE0003088FFF74BFF03000E20002B08D05E6872
:10ACF000002E05D021002800039B029A0097B04740
:10AD000007B0F0BD0A4B10B5984207D101220023CD
:10AD100052420A808B708A808B7110BDFFF73CFF16
:10AD20000028FAD001235B42038000238370F4E7FC
:10AD3000FFFF0000F8B5050001290AD1134E0024D9
:10AD40003388F227AB4219D028001149FFF7DAFF08
:10AD500006E0022904D10139FDF750FF0028EDD0AB
:10AD6000F8BD3B0063437268D018D35A002B09D05A
:10AD70003A00002100F0ECFE0134E4B2054B1B78F0
:10AD8000A342EED801235B423380DDE7646BFF1FF3
:10AD90007C68FF1F626BFF1F10B5FFF7FDFE03000D
:10ADA0000020834200D0987810BD0000F0B589B033
:10ADB0001C000EAB80CB03901E8810AB1B78049256
:10ADC00002930B7A0D00DB0616D42B780593022B29
:10ADD00024D00498FFF7D2FE002812D003689C46C6
:10ADE000002B0ED0029B2200019329003B006446F9
:10ADF00003980096A04705E00498FFF7BFFE0028DF
:10AE000002D10E2009B0F0BD8368002BF9D00A22D0
:10AE10002900039898470028D7D0F3E76B68587843
:10AE20001A786B4B000210439842D2D8043B9842E8
:10AE300010D2684B984242D015D8674BC0180128F1
:10AE4000C7D80B20002EDDD1EB681A7859683A80FC
:10AE5000200028E0614BC018032800D979E000F0F9
:10AE60000FFF846A789E5E4B9842B2D10B20002E71
:10AE7000C8D101233B80EB6831001B7823706889BF
:10AE8000013080B2FCF7A2FF3A88031E0ED0017891
:10AE900002328A183A80428962704289120AA2708C
:10AEA00059680278E01C00F00BFF06E004323A809B
:10AEB00031000422601C00F04BFE0020A2E70B20B2
:10AEC000002E9FD1EB6807A91E8804233B80330A1C
:10AED000300026706370FCF779FF051E28D004ABA4
:10AEE0009A890E2304A95B183E49C668FCF7E2FF65
:10AEF00000280BD12B783C486A680599FBF798FB32
:10AF0000002803D1012304AA5B42D3813278022AAC
:10AF100006D17168201D00F0D3FE3B8802333B80D0
:10AF20000E2304AA9B181B88A3701B0AE370C4E7B6
:10AF300004ABDE81F4E70B20002E00D062E7E96865
:10AF40000398FFF729FF02233B802070000A6070FE
:10AF5000B3E70B20002E00D054E70222EB681B88D9
:10AF60003A8023701B0A6370A7E7E86800F020FEB0
:10AF7000C2B203000720B24200D243E70DD00299CB
:10AF8000DBB27118994202DB921BD3B20293029B8F
:10AF9000E9681A003B8089195AE70023F6E70B207D
:10AFA000002E00D02EE70722EB683A801A78227034
:10AFB0005A7862705A88A2705A88120AE2701A7916
:10AFC0002271DA886271DB881B0AA37175E7C046BB
:10AFD000042900000228000000D8FFFFFFD6FFFF71
:10AFE00003280000FFFF000064C00011F0B58DB021
:10AFF0006B460020089120229B5E83423DDAA64BDF
:10B00000187800F05DFD071E32D00378B02B2CD1EC
:10B010000079023816281FD800F0E2FE17001E0043
:10B020001E001E0031001E0096001E001D011E00A5
:10B0300052011E0073011E00CD011E0050021E00B1
:10B040001E001E008E021E00E302944B94491B88D2
:10B0500078880B80FBF72CF83800FCF7ADFF914B9C
:10B060001B68002B01D038009847380000F0C0FB67
:10B070008020089B0002434018000DB0F0BDEE2276
:10B080000021874800F064FD0BAA3B7B7989388951
:10B0900000923A000D32FCF7B1FD0400804B1B78A2
:10B0A000002C3FD146E0804B788805937F4B4100D0
:10B0B000CB5A0BAE073BDBB23288029300230193DD
:10B0C0007B4B210006930093059BFFF76FFE744DA9
:10B0D000002810D1069B3A8A1B889A420BD138006F
:10B0E0000599123000F05CFD002804D02B786289AD
:10B0F0009B00EB185A80162306A81B1832882000E4
:10B100007989FCF7D7FE2B7804009A00AA18518899
:10B110000029C3D00133DBB22B70002807D006A969
:10B12000C98A9180634A12889A42BCD802E0012100
:10B1300049429180002B04D059497888FAF7ECFFF6
:10B140008AE73E890A2479E000253E89574B069319
:10B150007B88069A5B009B5A033B9D4202DB002DD5
:10B16000F0D05BE0162206A812183B7B798900928A
:10B170003A0030000D32FCF741FD0590002858D010
:10B180004689017A7888FCF703FD041E44D1464BBA
:10B1900078880793069B4100C95A454B0439C9B2C8
:10B1A00006AAD28A06930291019400930599079BFF
:10B1B000FFF7FCFD041E2FD1069B39491A88931C0A
:10B1C000002D26D14B807988384B4900CB5A511934
:10B1D000033B8B4220DD059B31485B8941190B7194
:10B1E000A91C0135C9B2EDB2059145191B0A2B7195
:10B1F000059B2D490433181800F062FD2C4B059A6D
:10B200001B88D318DDB22C4B9E4205D00136B6B256
:10B210009CE749889942D6D0002D0CD0204C2800BC
:10B22000618800F01DFB207021007888FAF784FF08
:10B2300012E7059CF0E7002C00D183E77B78142B04
:10B2400000D109E716493B794E800B700C71788864
:10B25000FAF724FF00E7162406ABE418210038892A
:10B26000FCF7B4FD011E00D1B7E1788822880F4CAD
:10B2700045002C5B0A4D013CE4B2029400240F4BC4
:10B2800001940095FFF792FD041E00D014E12900FF
:10B290007888FAF761FFDFE66C6BFF1F2443FF1F1E
:10B2A0008468FF1F7868FF1F7869FF1FB464FF1F61
:10B2B000686AFF1F2243FF1FFFFF00008668FF1F11
:10B2C000162406ABE41821003889FCF77FFD011E27
:10B2D00000D182E178882288AE4C45002C5BAE4DCF
:10B2E000013CE4B202947C89AC4B01940095FFF7D9
:10B2F0005DFD041E00D0DFE029007888FAF736FFF4
:10B30000AAE60025A44B1D803B00F6331B78A24A19
:10B3100078880792AB4208D99E4B1288069306990B
:10B3200043005B5A013B9A4203DB0799FAF728FF77
:10B3300092E616246B00FB18059306ABE418059BF8
:10B3400021001889FCF742FD011E03D1059B012451
:10B350001E8973E77888924B2288069C09934300E4
:10B360001B5B904E013BDBB20293002300960193DE
:10B37000099BFFF71BFD041E02D0059B1E895DE79C
:10B380007B88069A5B009B5A079A108832881218AD
:10B39000934202DC1B1A013B33807F4C023032881F
:10B3A0000999001900F08CFC2388328801359B181C
:10B3B0002380EDB2A8E70BAA3B7B798938890092FC
:10B3C0003A000D32FCF71AFC00250590059B002B76
:10B3D00004D10A24002D00D16EE060E0059B78883E
:10B3E000197AFCF7D5FB0100041E63D1694C6C4B44
:10B3F000788806940993069B4400E45A694B063CFE
:10B40000E4B20BAE32880793029401910093059940
:10B41000099BFFF7CBFC041E4CD1079B5E491B88A0
:10B420001A1D002D30D14A80059B5B4C5A89631947
:10B430001A716B1C9BB2E318120A1A71162306A824
:10B4400032881B1879890598FCF734FDFF21AA1C66
:10B450002E1D03350B00059092B2B6B2ADB2002896
:10B4600003D006ABDB8AD9B21B0AA2186519117189
:10B470002B714C4D301D2A884949201800F020FCC2
:10B480002B88F618B5B2A1E74988914207D17A888E
:10B4900006995200525AEB18053A9A42C4DC3E4CC7
:10B4A0002800618800F06CFC207021007888FAF791
:10B4B00071FED1E5002DF2D13E89BFE6162606AB1E
:10B4C000F61831003889FCF781FC3D000400FA359C
:10B4D00000282DD0037A9B060CD400227B89398961
:10B4E000788800923A000C32FFF7E8FB041E10D077
:10B4F0003E8915E03088FFF741FB00281AD08368A9
:10B50000002B17D02100122278889847041EE4D01F
:10B51000EEE72B78002B02D17888FAF74BFE002655
:10B520002B78002B00D097E5002C00D194E585E620
:10B530000124DDE70E24DBE7162506ABED18290014
:10B540003889FCF743FC041E47D0037A9B0611D4CC
:10B55000154A7B881188994203D01448814207D14B
:10B560001380134BF2261D780023D9B2A94221D3B0
:10B570000924A1E72888FFF701FB00282FD0836862
:10B58000002B2CD02100122278889847041EDFD08F
:10B5900092E7C046B464FF1F8468FF1F8668FF1FE0
:10B5A0007869FF1F686AFF1F646BFF1FFFFF0000C1
:10B5B000626BFF1F31005943546801336018615AB0
:10B5C0000029D2D13C0008342100F22200F078FB9F
:10B5D00021007888FAF7F6FD3EE501246CE70E2499
:10B5E0006AE71D4B1A887B889A4231D07888FAF72F
:10B5F000F3FD31E5F223059851684343CD18C95A4C
:10B6000000291FD03B7A012B0BD16C88AB8878883E
:10B61000AA1D0094FFF752FB041E02D000233B72C8
:10B620002E88F2220021280000F092FA00232B80BD
:10B63000059B0133DBB20593084B05991B78064A3D
:10B640008B42D7D801235B421380002CCED0F5E586
:10B65000002634000596EFE7646BFF1F626BFF1F47
:10B6600070B504000E001500FFF796FA031E08D10E
:10B6700031000548FFF790FA03001120002B02D09B
:10B680001C8000209D7070BDFFFF0000F8B50B4FBF
:10B6900006003B780D001400FF2B0ED00A2000F0AE
:10B6A00097FB011E09D0B12303800023468003715C
:10B6B000C5800481387800F093F8F8BD7944FF1F05
:10B6C000F7B50F0008A90600088809A90B24098806
:10B6D000002821D10234022B1ED1557813782D0277
:10B6E0001D432B008B4301937334002B14D1FB6853
:10B6F000300019000093FFF74FFB019C85420BD0EF
:10B700002A0030000099FFF7ABFF041E04D12A0085
:10B7100030007989FFF7BAFF2000FEBDF0B50E7842
:10B7200085B003900AA805880120022E0DD14C682F
:10B730002778647824023C43054FBC4205D1039826
:10B74000DBB201960095FFF7BBFF05B0F0BDC04628
:10B7500002290000034B10B51B68002B00D098474E
:10B76000FEE7C046706BFF1F07B501A8FFF7F2FFA9
:10B77000044A05480021121A00F0C2F8F8F77CF8D4
:10B78000FEE7C046746BFF1F7C44FF1F00000000F3
:10B7900001B40248844601BC604700BF3133FF1F3B
:10B7A00001B40248844601BC604700BFA536FF1FB4
:10B7B00001B40248844601BC604700BF8D39FF1FB9
:10B7C00001B40248844601BC604700BF9936FF1FA0
:10B7D00001B40248844601BC604700BF091B000059
:10B7E00001B40248844601BC604700BF594F0100C4
:10B7F00001B40248844601BC604700BF434D0100CC
:10B8000001B40248844601BC604700BFADAE0000F1
:10B8100001B40248844601BC604700BFF30E00003B
:10B8200001B40248844601BC604700BF5131FF1F8C
:10B8300001B40248844601BC604700BFD11BFF1F12
:10B8400001B40248844601BC604700BF11470100B3
:10B8500001B40248844601BC604700BF01240000D7
:10B8600001B40248844601BC604700BF350E0000A9
:10B8700001B40248844601BC604700BF8B520100FE
:10B8800001B40248844601BC604700BF4551010035
:10B8900001B40248844601BC604700BF2526000071
:10B8A00001B40248844601BC604700BF5522000035
:10B8B00001B40248844601BC604700BFCD39FF1F78
:10B8C00001B40248844601BC604700BF712EFF1FCF
:10B8D00001B40248844601BC604700BF9DA9000036
:10B8E00001B40248844601BC604700BFF94C010026
:10B8F00001B40248844601BC604700BF6134FF1FA9
:10B9000001B40248844601BC604700BFB70E000086
:10B9100001B40248844601BC604700BF21240000F6
:10B9200001B40248844601BC604700BF4D38FF1F88
:10B9300001B40248844601BC604700BF3919FF1FAB
:10B9400001B40248844601BC604700BF2951010090
:10B9500001B40248844601BC604700BF011AFF1FC2
:10B9600001B40248844601BC604700BFE1170000F3
:10B9700001B40248844601BC604700BF5D17000067
:10B9800001B40248844601BC604700BFF132FF1F8A
:10B9900001B40248844601BC604700BF4550000026
:10B9A00001B40248844601BC604700BF59520100FF
:10B9B00001B40248844601BC604700BFC9260000AC
:10B9C00001B40248844601BC604700BF311B00003F
:10B9D00001B40248844601BC604700BFB130FF1F7C
:10B9E00001B40248844601BC604700BF691F0000E3
:10B9F00001B40248844601BC604700BF055E0000F8
:10BA000001B40248844601BC604700BF6DBC000021
:10BA100001B40248844601BC604700BF0D19FF1FF6
:10BA200001B40248844601BC604700BF851F000086
:10BA300001B40248844601BC604700BF9937FF1F2C
:10BA400001B40248844601BC604700BFB352010004
:10BA500001B40248844601BC604700BFF53AFF1FAD
:10BA600001B40248844601BC604700BF3555000060
:10BA700001B40248844601BC604700BF8552010002
:10BA800001B40248844601BC604700BF65710100F3
:10BA900001B40248844601BC604700BF5539FF1F0E
:10BAA00001B40248844601BC604700BFC936FF1F8D
:10BAB00001B40248844601BC604700BF350E000057
:10BAC00001B40248844601BC604700BFF54E010046
:10BAD00001B40248844601BC604700BFED4A010042
:10BAE00001B40248844601BC604700BF493BFF1FC8
:10BAF00001B40248844601BC604700BFD949010037
:10BB000001B40248844601BC604700BF21460100E1
:10BB100001B40248844601BC604700BF793AFF1F68
:10BB200001B40248844601BC604700BF0D520100C9
:10BB300001B40248844601BC604700BF1D4B0100B0
:10BB400001B40248844601BC604700BFEDA5000077
:10BB500001B40248844601BC604700BF154D010096
:10BB600001B40248844601BC604700BF291C0000A4
:10BB700001B40248844601BC604700BFC56D0100A6
:10BB800001B40248844601BC604700BF554901002A
:10BB900001B40248844601BC604700BFC930FF1FA2
:10BBA00001B40248844601BC604700BFCD4C01008F
:10BBB00001B40248844601BC604700BFDD52010069
:10BBC00001B40248844601BC604700BF090E000072
:10BBD00001B40248844601BC604700BF3D4B0100F0
:10BBE00001B40248844601BC604700BF213BFF1FEF
:10BBF00001B40248844601BC604700BFC51D000077
:10BC000001B40248844601BC604700BFB14E000049
:10BC100001B40248844601BC604700BF51250000C2
:10BC200001B40248844601BC604700BF156B0100A7
:10BC300001B40248844601BC604700BFE928000007
:10BC400001B40248844601BC604700BFD91B000014
:10BC500001B40248844601BC604700BF653BFF1F3A
:10BC600001B40248844601BC604700BFA9460100F8
:10BC700001B40248844601BC604700BFB54C0100D6
:10BC800001B40248844601BC604700BF793BFF1FF6
:10BC900001B40248844601BC604700BFDD66010074
:10BCA00001B40248844601BC604700BF75A900008A
:10BCB00001B40248844601BC604700BF056A000029
:10BCC00001B40248844601BC604700BFE94C010052
:10BCD00001B40248844601BC604700BF014C01002A
:10BCE00001B40248844601BC604700BF4D1F0000FC
:10BCF00001B40248844601BC604700BF017F0000D8
:10BD000001B40248844601BC604700BF8D120000A8
:10BD100001B40248844601BC604700BF514701009E
:10BD200001B40248844601BC604700BF0D3AFF1FC2
:10BD300001B40248844601BC604700BF7918000086
:10BD400001B40248844601BC604700BFE5480000DA
:10BD500001B40248844601BC604700BFC9A9000085
:10BD600001B40248844601BC604700BF3D18000092
:10BD700001B40248844601BC604700BFA54F0100E2
:10BD800001B40248844601BC604700BF090E0000B0
:10BD900001B40248844601BC604700BF456B010006
:10BDA00001B40248844601BC604700BF4139FF1F0F
:10BDB00001B40248844601BC604700BFC94A010083
:10BDC00001B40248844601BC604700BFC5210000A1
:10BDD00001B40248844601BC604700BF1D4D01000C
:10BDE00001B40248844601BC604700BF8D3BFF1F81
:10BDF00001B40248844601BC604700BF810E0000C8
:10BE00000003010302020303040205000602070007
:10BE1000080009020A030B030C000D000E030F03B8
:10BE2000100311031300140015031603453C001101
:10BE3000793C0011000000000200000042BE001129
:10BE4000192A0F180A000000F1590000FD24000013
:10BE500041460100098200111DA2001171760011F6
:10BE60000D80001149540011EDAF001195500011E3
:10BE7000553E0011853F001100000000161600001D
:10BE8000020000008CBE0011F4FFF3FFD2FC0000A2
:10BE9000C5400011000000000000000054757961E9
:10BEA0000042322E300030303138006769746875D6
:10BEB000622E636F6D2F707676780054483035446B
:10BEC0000000000002000000D8BE0011292A282A24
:10BED000272A262A252A242A0A180000E20400001C
:10BEE0007102000078EC00000500000074400000C2
:10BEF0001027000060F0000004000000066400004D
:10BF0000204E000000000000060000005C4400001D
:10BF1000102700006CEE0000070000000500000084
:10BF20001F501D10023CB40000011800200000004A
:10BF3000A1020000303132333435363738394142CE
:10BF400043444546000000004D580011A15800111F
:10BF5000000000000200000060BF00116F2A6E2A7E
:10BF60001A18EAD8BC80F0FC600000000000000055
:10BF700000005F066B2F363D7D077F3F777C596E53
:10BF80007971AF066D4FC6CBEB0EEFCFEEC3A9664E
:10BF9000E9E8FA60D6F46CBCBEE0FEFCEE3E9A76B0
:10BFA0009E8E000001A00000000000006410B71D7C
:10BFB000C8206E3BAC30D9269041DC76F4516B6BD7
:10BFC0005861B24D3C7105502083B8ED44930FF099
:10BFD000E8A3D6D68CB361CBB0C2649BD4D2D3864F
:10BFE00078E20AA01CF2BDBDFB349B5F800000809C
:10BFF000001000000000000073620011FD780011C5
:10C0000097620011057D00111B630011DB7C00119C
:10C0100091630011B17C0011E3630011797E00117E
:10C020004B640011797E00117D640011337E001194
:10C0300091630011697C001109640011117E0011E7
:10C040000000000000000000EF640011117E0011EC
:10C050005165001115790011052A042A012A002AC8
:10C0600002290328012800280118001800000000F8
:10C070000000000000000000000000870101020134
:10C080000201010201020303040103010101010194
:10C090000303020103000D000E0010001100130045
:10C0A0001401070108010A010B011C011D02040211
:10C0B00005020702080219021A021C021D030103ED
:10C0C000020317000201000504000807000B0A0024
:10C0D0001716001D1C010201010504010E0D0111BE
:10C0E00010011413011716011A19020201020B0A9A
:10C0F000020E0D0211100214130217160305040399
:10C100000807030B0A030E0D0001020307090A0BBF
:10C110000E0F101112141718191A1B1F20212200BC
:10C1200035A90011F1A90011000000000200000073
:10C130006AC00011000000001DB7001100000000DF
:08C140000200000068C00011BC
:020000041FFFDC
:1000000000000000BD3D001148BE001144BE0011BB
:10001000AC61FF1F000000000000000000000000B5
:1000200000000000000000000000000000000000D0
:1000300000000000000000000000000000000000C0
:1000400000000000000000000000000000000000B0
:1000500000000000000000000000000000000000A0
:100060000000000000000000000000000000000090
:100070000000000000000000000000000000000080
:100080000000000000000000000000000000000070
:100090000000000000000000000000000000000060
:1000A0000000000000000000000000000000000050
:1000B0000000000000000000000000000000000040
:1000C0000000000000000000000000000000000030
:1000D0000000000000000000000000000000000020
:1000E0000000000000000000000000000000000010
:1000F0000000000000000000000000000000000000
:1001000000000000000000000000000000000000EF
:1001100000000000000000000000000000000000DF
:1001200000000000000000000000000000000000CF
:1001300000000000000000000000000000000000BF
:1001400000000000000000000000000000000000AF
:10015000000000000000000000000000000000009F
:10016000000000000000000000000000000000008F
:10017000000000000000000000000000000000007F
:10018000000000000000000000000000000000006F
:100190005533FF1F9D31FF1FC166010000000000A5
:1001A000000000000000000000000000000000004F
:1001B000000000000000000000000000000000003F
:1001C000000000000000000000000000000000002F
:1001D000000000000000000000000000000000001F
:1001E000000000000000000000000000000000000F
:1001F00000000000000000000000000000000000FF
:1002000000000000000000000000000000000000EE
:1002100000000000000000000000000000000000DE
:1002200000000000000000000000000000000000CE
:1002300000000000000000000000000000000000BE
:1002400000000000000000000000000000000000AE
:10025000000000000000000000000000000000009E
:10026000000000000000000000000000000000008E
:10027000000000000000000000000000000000007E
:10028000000000000000000000000000000000006E
:10029000000000000000000000000000000000005E
:1002A000000000000000000000000000000000004E
:1002B000000000000000000000000000000000003E
:1002C000000000000000000000000000000000002E
:1002D000000000000000000000000000000000001E
:1002E000000000000000000000000000000000000E
:1002F00000000000000000000000000000000000FE
:1003000000000000000000000000000000000000ED
:1003100000000000000000000000000000000000DD
:1003200000000000000000000000000000000000CD
:1003300000000000000000000000000000000000BD
:1003400000000000000000000000000000000000AD
:10035000000000000000000000000000000000009D
:10036000000000000000000000000000000000008D
:1003700069B700110000000000000000000000004C
:10038000000000000000000000000000000000006D
:10039000000000000000000000000000000000005D
:1003A000000000000000000000000000511BFF1FC3
:1003B000000000000000000000000000000000003D
:1003C000000000000000000000000000000000002D
:1003D000000000000000000000000000000000001D
:1003E000000000000000000000000000000000000D
:1003F00000000000000000000000000000000000FD
:08183800806FFF1F4118FF1F24
:10184000024981F3088802F053FB0000806FFF1FFC
:1018500070B500241E491F4A1F484C6308CA1B0567
:101860001B0DE4188242F9D11C4B80228B630021AE
:1018700009201B4B920519621A4B1B4DDA671B4B53
:10188000DA688243DA609A68194802409A60112047
:10189000296002F0BBF8112002F098F86B6C154A31
:1018A000112013406B64144B144A63431B0C1384C4
:1018B0000122134B9A7201F027FC124B1B78002B6C
:1018C00004D1114B1021187802F002FB70BDC04604
:1018D000000005408807054000080540FF010000A2
:1018E00000F0004004E100E0003800403CF000401F
:1018F000FFDFFFFFFFFDFFFFAE0600007C61FF1F63
:101900003062FF1F5E64FF1F5C62FF1F10B502F0B4
:101910004FF9072804D0122808D0022808D010BD9B
:10192000044A0420136B01331363F8E70220F6E73F
:101930001420F4E75C65FF1FF8B507000C002600D3
:101940002500503630785135002804D10300287026
:1019500058342370F8BD2978CA00481E8141A31865
:101960003800A25C5B68C9B2FFF7D0FF00280DD138
:101970002B78DA00A218013350602B703378044AB8
:10198000013B3370136A01331362D8E70123DFE7A9
:101990005C65FF1F5C234343074910B5C9180B0062
:1019A00058331B78012B05D1FFF7C6FF034A936A12
:1019B0000133936210BDC0469065FF1F5C65FF1F39
:1019C00010B502F00DFA064A0121130010CB49426E
:1019D000D967044B136002F07BF9200010BDC046AC
:1019E00000E100E01000100010B5040002F0F8F96A
:1019F000024B1C6002F06CF910BDC04600E100E033
:101A000010B5040002F0ECF94021094A20001368E7
:101A10008B43136000F0F6FA01F07EFC0022054BC8
:101A200001201A60044B04321A6002F011FAFEE73A
:101A30001CF00040C4F00040C0F00040431E5A4279
:101A40005341A022F0B5D2015B421340154D164A16
:101A500040019B182A18127E8BB00191002A1BD0DE
:101A60001A000832D46F0022E6B206AFE4B2944204
:101A70000EDC2818C369002B08D0019902AA117145
:101A800006AA049202AA167303A898470BB0F0BDE9
:101A90001978B9540132EAE71A7D1A7806AB0126A3
:101AA0001A70E6E71C68FF1F00400040F0B5254BA8
:101AB00004004001C25C85B0002A2BD01A18117EA8
:101AC000002927D0917E002924D01179022921D123
:101AD0001689D788D168F51BADB22A1C102D00D904
:101AE000102292B2BE4217D11818012303710023AD
:101AF000C269C38003819A4206D0684603210373FA
:101B00000171029301A890470820002C00D01920F1
:101B100001F0FAFA05B0F0BD013C65426C41A02528
:101B20006442ED012C40084D1B186419074D063323
:101B3000013A92B2AA42EDD01888461C1E80085C79
:101B40002070F5E71C68FF1F00400040FFFF000009
:101B50000F220E4B10B59868104002380A280BD897
:101B600002F00AF80D0A0B0A0A110A0A0A0A06000C
:101B700002210020FFF762FF10BD0121F9E70020DC
:101B8000FFF794FFF8E7DB6FF6E7C0460040004040
:101B90000F220E4B10B59868104002380A280BD857
:101BA00001F0EAFF0E0A0B0A0A120A0A0A0A0600E4
:101BB00002210120FFF742FF10BD01210800F9E7D3
:101BC0000120FFF773FFF7E7DB6FF5E700900040B8
:101BD00013B5334C2378072B3DD8324B1A78324B50
:101BE000002A39D18022196852020A431A6025203E
:101BF00001F0CCFE20232D4A11680B438021136095
:101C00006B460422C90508680733104228D080219A
:101C10000422C905C86810422ED080212020C905A1
:101C2000CA688243CA6014221A701A78002A2FD117
:101C30008021C905C86820320243CA6014221A7084
:101C40001A78002A28D11A4B1A7D22785A601D2250
:101C50001A705932DA6013BD1A6816490A40C5E78E
:101C6000086802430A6014221A701A78002ACED03B
:101C70001A78013AD2B2F7E7C8680243CA60142260
:101C80001A7019784A1ED2B21A700029F9D1C4E725
:101C90001A78013AD2B2C7E71A78013AD2B2CEE73F
:101CA000B443FF1F7C44FF1F3CF00040AC43FF1FC8
:101CB00000200040FFFFFEFF564B70B51B68012B54
:101CC00003D1554A936D0133936501F0C9FF534B1E
:101CD000534A1860534B544C1A600123534A136003
:101CE000534A13602378002B06D0062251495248EC
:101CF00002F07EF900232370504A514B10681B7884
:101D0000C1B2002B0ED14F4CC0B223785BB2002B76
:101D10004FDB237824785BB264B21B0424021B19C6
:101D20001B1813600B1C50294ED95023464A4749B3
:101D30001078DBB2FF2202284BD10868444C454D95
:101D4000267890432A78964254D9227824782E789F
:101D5000023B5D10A31B6B435201D31A10335B117E
:101D60001843086002F024F9031F012B45D83A4BB1
:101D70001B78002B06D0394B1B78002B02D000209B
:101D800001F00EFFA122364B92009978354B4A4361
:101D90001B689B18832292009B181B78033B012B26
:101DA00003D8AF20400002F003F801222E4BDA8264
:101DB00070BD237824785BB264B2FF33FF341B0418
:101DC00024021B190138ABE7CAB2022AAED20223A1
:101DD000ACE70868254C264D267890432A78964231
:101DE00008D9227824782D78023B5B10641B63436A
:101DF0005201B2E72378DBB2B2E70228D5D11D4BFE
:101E00001B78013B022B03D91B4B1B78022BCCD137
:101E10006C20C8E79809FF1FFC0FFF1FA864FF1F75
:101E2000FF3F000014100340AC64FF1F0C10034080
:101E300000100340D50BFF1F7211FF1FB4000340B9
:101E40008C09FF1F680AFF1F490AFF1F9400034007
:101E5000460AFF1F470AFF1FF908FF1F2209FF1F3D
:101E6000300DFF1F3409FF1FBC0BFF1F440AFF1F6B
:101E7000450AFF1F1C09FF1F2309FF1F10B502F0B1
:101E80003FF80022014B1A8010BDC046A664FF1F18
:101E900010B501F0EDFFA121054A89009478054AAB
:101EA00061431268044B5218528C1A8010BDC04610
:101EB000300DFF1F3409FF1FA664FF1F10B50D4B27
:101EC0000D4A9978A1239B004B431268D218531DE9
:101ED000D97F0A4B1B88994209D2441C07D0C828D5
:101EE00005D0D2695B1A5A43054B5343C01802F020
:101EF000B7F810BD300DFF1F3409FF1FA664FF1F88
:101F00007102000070B5244D2B68002B28D002F020
:101F10000FF82B68D8402B680400002B27D001F065
:101F2000B7FF2B68D8401D4B1D4A9978A1239B0011
:101F30004B431268D118D25C91239B00002A20D019
:101F4000CA580132CA50174B17491B6808688342A8
:101F500014D3D23B181A012A1AD0144B186070BD42
:101F600001F0E6FF124B196802F09AF8D3E701F08E
:101F70008FFF0F4B196802F093F8D4E70D495B18F7
:101F8000E8E7CA500C4B1B68DB68E418201AE4E74A
:101F9000F530FF30E1E7C0461C08FF1F300DFF1F82
:101FA0003409FF1F9C09FF1FA864FF1FA009FF1F22
:101FB0001808FF1F2DFF3F00B064FF1F70B504001D
:101FC0000D00282916D10300A433C2881B889B1A50
:101FD0000B4A9BB293420DD906006A3605223100A6
:101FE000653001F055FE002804D13100200001F0D9
:101FF00007FF70BD2900200001F0CAFFF9E7C046C5
:10200000FE7F0000F8B50500012001F089FE134CA9
:10201000A36AA26A9342FBD1114E336001F0F8FE2D
:102020001049030008601048426894460F4A176838
:102030000022BC4501D24268BA1A0D4802603268DB
:10204000AD18A422E562606A520302436262094A43
:102050001278002A01D00F3B0B60F8BD00F0004061
:10206000340AFF1FE408FF1F28100040180AFF1F52
:102070001C0AFF1F1C09FF1F70B580241025E405F2
:10208000A3682B43A36001F01BFFA368AB43A360CD
:1020900070BD0000F7B5160080221C001023D20589
:1020A0000191916805000B43936000225A4BD73091
:1020B0001A6001F02DFE9D232A002F009B00EB5893
:1020C000CA3201210092FC37002B01D00021009A76
:1020D000386801F0B5FD2900009BCB311A784F4BD1
:1020E000D3351A604B780A781B0213438A7812049E
:1020F0001A43CB781B061343494A1BBA13604B792A
:102100000A791B0213438A7912041A43CB793100EE
:102110001B061343434A1BBA13606B782A781B02D1
:102120001343AA7812041A43EB781B0613433E4A62
:102130001BBA1360019A330213433C4A13603C4BB1
:1021400022001B1B9C4603293DDCB3089A001300A8
:102150005142B21A032A46D1354AE018511A827800
:102160004078120400020243E05C043302430A6038
:102170000022FF2B4BDDF0222E4B12011A600F22A2
:102180002D4B1A602D4A1368002BFCD00023224AE5
:1021900027491360091B321D0B191B68043A180AE2
:1021A00023706070180C1B0EA070E3700434002ABA
:1021B000F2DC802210213B68D20501333B6093683A
:1021C0008B439360F7BD6346D578981893782D06B6
:1021D0001B042B43157804392B43557804322D0208
:1021E0002B430360AFE7022A0AD1114AE05C511A7F
:1021F000E2185278120202430A6004339BB2B7E736
:10220000012AB5D10A4A521AE15C1160F5E7084982
:1022100059180A600433ACE7000004403C00044055
:102220003800044034000440300004400C000440F6
:102230000001044004000440100004401400044065
:10224000F7B5150080221C001023D205009191687B
:1022500007000B4393600023654AD730136001F0F9
:1022600057FD9D233E009B00F9583B00CA363200C3
:10227000FC33002900D07FE0586801F0E1FC390010
:1022800032785C4BCB311A604B780A781B021343CF
:102290008A78AC4612041A43CB78281D1B061343D8
:1022A000554A1BBA13604B790A791B0213438A798A
:1022B00012041A43CB791B061343504A1BBA13600E
:1022C0004B7A0A7A1B0213438A7A12041A43CB7A96
:1022D00021001B0613434A4A1BBA1360009A2B02C3
:1022E0001343484A13602200474B1B1B0093009B7B
:1022F000CE785B1801938B7836061B0433430E7837
:10230000043833434E78043136023343019E336040
:102310000328ECDC0321A808431C9B002940800013
:1023200003292BD13849E5185E18A9786D78E35C4C
:1023300009042D02294319433160030008330021A9
:10234000FF2B2DDD314B324919600F21314B1960C4
:10235000012327490B60304B19680029FCD0062166
:102360001B680B40042B20D080220020D2059368EC
:102370000A318B439360FEBD01217DE7022908D11C
:1023800021495D18E1184978E35C09021943296085
:10239000D3E70129D3D11C495918E35C0B60CCE782
:1023A0001948181801600433CAE7002310490B606C
:1023B0006346002B0CDC3B00FC335A6810210132D1
:1023C0005A608022D205936801208B439360D2E744
:1023D000009B9B181B68190A13705170190C1B0E77
:1023E000D37004235B4291709C440432E0E7C04602
:1023F000000004403C000440380004403400044025
:10240000300004400C00044000010440040004407B
:10241000080F0000100004401400044070B5061EB0
:1024200019D002225A4B9B799343012B13D1594B5C
:102430001A78FF2A0FD15A78FF2A0CD19A78FF2AEE
:1024400009D1DA78FF2A06D11A79FF2A03D15B79FC
:10245000FF2B00D199E0504B0C201A78012A08D0AC
:1024600000224E4D1A7029780B00093B042B01D82D
:10247000212070BD4B1F012BFAD9454CA37B042BA7
:1024800000D982E0A279032A00D97EE09A1ED2B256
:10249000012A02D860881F2877D9002E56D0012E35
:1024A00073D1A0880128E3D0002907D1581E032842
:1024B00003D801F061FB121715122E702978481EFF
:1024C000032811D80025364B1D602823237501F001
:1024D0008FFCA84227D0A580CAE702212970EDE72A
:1024E0000421FBE70321F9E707390129C0D82D4969
:1024F0000968C96A8906BBD52B4908780028B7D175
:10250000012A01D9002BB3D102230B708021274D62
:10251000263389012878237501F052FC8021287820
:10252000890101F0D5FC0123A380214B1B78002BEE
:102530000AD0FA2280211F4B92001B8809025A43BD
:102540001A4B187801F004FC002092E701F048FCD7
:102550002B78A680073B012B03D917482E7001F07A
:10256000EFFB114B114C1A78002A06D08021002273
:10257000207889011A7001F023FC01F0A9FB802169
:102580002078090201F01CFCDEE7122071E7C0464A
:10259000A60BFF1F6B09FF1F1A09FF1F1C09FF1F56
:1025A0004809FF1FB064FF1F2309FF1F1B09FF1FFE
:1025B0002109FF1F2C09FF1F0010004010B5002942
:1025C00001D001F0CDFB10BDF7B5604B01919978BA
:1025D000A1239B004B435E4A060014681022E418B6
:1025E000D6235B00E0583623FF33E35C0027934398
:1025F000222B41D1574B0F3A1A600760012501F099
:1026000027FD019B1880E8235B00E35C002B01D0D1
:10261000B34258DD0023504FFB70AD33FF33E35816
:102620001A68002A03D09B88DB439B071DD0382300
:10263000FF33E35C002B18D09B235B00E35C002B93
:1026400013D1D133FF33E35CB3420EDAA4235B0032
:10265000E15AE018090A023101F0E2FC23000122EC
:10266000FE33013E01351A87FA70E8235B00E35C14
:10267000002B2AD0A8B2FEBD03683D00002BBED0BF
:1026800081880430090A023101F0CAFCD6235B00BC
:10269000E3581F60B2E72300B133BA00FF33985804
:1026A000013781880430090A023101F0B9FCE823BE
:1026B0005B00E35CBB42EEDCE822F61AED18002377
:1026C0005200A354A6E70027F1E7200001F0A8FB81
:1026D00000281FD0002E1DDD73198826471901938D
:1026E000B600200001F004FB5A308000201840683A
:1026F000013581880430090A023101F091FC200083
:1027000001F066FBA3590133A351BD4202D0019BE6
:102710009D42E6D1114BE35C002BABD095239B008F
:10272000E35C002BA6D00E4BE15A0029A2D00D4A43
:10273000A35C994202D90133A3549BE700231A21D9
:102740002000A35401F074FB94E7C046300DFF1F36
:102750003409FF1F00140340E010FF1F5A0200005D
:10276000720200005E0200000D4970B54A6E0D4C09
:10277000D2038B69D20BA24206D80B4D0224AA4287
:1027800004D901F06DFB70BD02246442E21815000B
:102790007E2425402242F4D0A3432B438B61F0E7F3
:1027A00000F000400A200000FC1C0000F8B51D4BA2
:1027B0001D4F1A78002A10D1BA7B002A02D10132AB
:1027C0001A7003E0032AFAD0022AF8D001F010FBB5
:1027D00000220120154B1A70F8BD154B154D1C68D1
:1027E000154B9E7801232B702878C0B200F09EFB19
:1027F000BB7B002B0BD101F053FBA1239B00734348
:10280000E41883239B00E41823782B70E4E7032B60
:1028100002D101F0B5FAF0E70020022BDCD101F083
:102820008FFBEAE71C09FF1FA60BFF1F2309FF1FF1
:102830003409FF1F490AFF1F300DFF1FF0B587B095
:102840000EAD2F780FAD2D780593AC46634614007E
:102850000E4D0CAA12782E7803930D9B00920193D3
:102860002200059B029701F053FB2E70012C01D032
:10287000042C08D1802206498B889343054A12789C
:10288000D20113438B8007B0F0BDC0461C09FF1F67
:102890006C11FF1F7809FF1F0B001B3B70B5040074
:1028A0003020E02B0DD81300E025493BFF3B9BB2C5
:1028B000ED00AB4205D8034B200019825A8201F08B
:1028C0001FFA70BD8410FF1F10B501F0C9F9054B48
:1028D00000205B68052B04D9034A5268D20200D459
:1028E000980810BD00100040FCE100E070B501F058
:1028F00077FA0D4B1B68FC33DC691D6AFFF7E4FFB8
:102900006419844204D2094B01241B68002B07D0B0
:1029100004220024064B1A70064A9369013393611E
:1029200001F0D6F9200070BDB064FF1F9809FF1FA9
:102930002309FF1FFC0FFF1F70B50C4D2B68FC33E4
:102940005C6A01F04DFAFFF7BFFF2B680025FC33EE
:102950009B6AE318834204D2054B1B68AB4200D14B
:10296000051B01F0B5F9280070BDC046B064FF1F1B
:102970009809FF1FD722044B92009B5810B5002BDB
:1029800000D0984710BDC0460000FF1F10B501F0F1
:10299000DBF8FFF7EFFF2749274BCA6D274C1A409A
:1029A00084235B001343CB65254B1B68186A01F039
:1029B000B7F9244B244A1A60244B254A1A60A022F6
:1029C000244B52001A60244B187801F039FB200088
:1029D000224901F015F90023A3600233A360204BC4
:1029E0002049236003232048A36001F009F9102245
:1029F0001E4BFF201A60802252031A60802292032D
:102A00001A60802212041A6001F0CAF8012001F055
:102A10009FFAFA20400001F0C3F9582001F0C8F9EC
:102A2000134801F04DF9012001F00AFA072001F0E6
:102A3000FFF810BD00F0004000FEFEFF1410004043
:102A4000B064FF1F000003400180063DBC0003404E
:102A500034080000A40003404A0AFF1F710200006E
:102A6000C3090000FFFF3F002810004000E100E024
:102A700030750000674E336888331B6883F308881D
:102A800001F0FEF9644A6549136800200B401360A9
:102A9000634B644A1B68934200D1A6E001F0A8F89A
:102AA0000221614A13688B431360FFF76FFF5F4B8E
:102AB0005F4C1878C0B201F0BBFA0023A360023368
:102AC000A3605C4B0120236001F02AF90323A3607B
:102AD00001F086F8040001F0C3F8050001F080F869
:102AE000554B186001F044FA544B1968621A531E92
:102AF000A14200D213008022D203934201D39B0251
:102B00009B0A3268D16AC90700D471E04C491C0C99
:102B100009689BB24C4359432402090A64180326EE
:102B20004849FC3293680A6847489B1A474A076835
:102B3000126847499B18474A9A1833409208DB1994
:102B40000A600360042B03D9013233400A6003603A
:102B50000E684149A619300001F0A2FA3F4F3E49E4
:102B60003B68C3183B603000019301F009FA3C4E0A
:102B70003068081838493060884205D9019B013314
:102B80003B6001F0FDF9316001F072FA354B1B78C2
:102B9000002B0DD001F064F8334B621B196812183A
:102BA0008A4232D24919091B091A304801F028F823
:102BB0002F4E337A002B0ED001F052F8621BF168D1
:102BC0001218914224D94919091B091A294801F000
:102BD00017F800233372284B83F3088801F020F89C
:102BE000002001F005F801F0A3F801F001F85CE71E
:102BF000DC0199000234641A5900641A09214B431C
:102C00008033CB40A408E41889E7FA218900CCE797
:102C10001A49DBE7B064FF1F1CF00040FFFFC1FF53
:102C20000C0AFF1FB641210310000040490AFF1F94
:102C300014100040C3090000100AFF1F340AFF1FD0
:102C4000380AFF1F200AFF1F280AFF1F1C0AFF1F48
:102C5000240AFF1FC4090000710200006008FF1F62
:102C60002C0AFF1F1C09FF1FE408FF1F0010004073
:102C7000740BFF1F3C10004000000020DC0500002A
:102C8000A022054B92009B5810B5002B01D098470D
:102C900010BD01F00DF8FBE70000FF1FA122054B5E
:102CA00092009B5810B5002B01D0984710BD00F042
:102CB000FFFFFBE70000FF1FA222054B92009B587D
:102CC00010B5002B01D0984710BD00F0F1FFFBE7D5
:102CD0000000FF1FA322054B92009B5810B5002B4C
:102CE00001D0984710BD00F0E3FFFBE70000FF1F95
:102CF000A422054B92009B5810B5002B01D0984799
:102D000010BD00F0D5FFFBE70000FF1F70B500F01D
:102D1000A7FF4F4B186000F0C3FF0400C30702D4A5
:102D200001F0DEF870BD00224A4B1A604A4B187859
:102D30000138042829D800F01FFF0320181C2400A4
:102D4000200001F0EDF80128ECD0444C2378042B4E
:102D50006ED101F0ADF80028E4D001F001F958205F
:102D600001F026F802232370DCE7200001F088F947
:102D7000E9E7200001F04CF9E5E7200001F010F947
:102D8000E1E7200000F044FFDDE701F011F9050064
:102D9000012808D1324B1B78053B012B03D82000BA
:102DA000FFF76EFFD1E72D4B1B78022B01D0052BCF
:102DB00020D1022D28D12B4B9B7BAB431CD1200073
:102DC000FFF76CFF264B18780128BED16405BCD4F0
:102DD000244925224B7B034205D1233A13405A4212
:102DE000534126331A000B7D9342AED9322000F0B6
:102DF00077FFAAE7022D07D1194B1B78052B11D1BC
:102E00002000FFF759FFDDE7012D0BD1012B03D186
:102E10002000FFF75FFF98E7062B03D12000FFF7A4
:102E200067FF92E7200000F043FF022D8DD1C9E734
:102E3000032B04D10C4B987C01F02AF972E7072B85
:102E400000D06FE7094B987B01F0C2F86AE7C046F3
:102E50009C09FF1F9809FF1F9009FF1F2309FF1FEF
:102E60001C09FF1FA60BFF1FBC0BFF1FD40BFF1F6E
:102E7000FA210A4B0A4A49001A640A4A5A500A4A75
:102E800004395A50094A08319A64094A5A50094A81
:102E90005C315A50084ADA667047C0460000FF1F8E
:102EA0003D28FF1F3929FF1FED28FF1F1D24FF1F8D
:102EB000AD27FF1FBD1EFF1F911EFF1FF7B50B0C97
:102EC000FF270122009300233C001E001D009446B2
:102ED000019089B262469A401000084018413618A5
:102EE000B6B2FF2F02D1012E00D19FB2009802404E
:102EF0001A41AD18ADB2FF2C02D1012D00D19CB208
:102F00000133102BE6D10320012E07D1012D04D16E
:102F1000019B2401E4191C700138FEBD102EFCD168
:102F20000238102DF9D00230F7E700008023F7B502
:102F30009C46264B264F01932649274A274D284C6D
:102F4000284B02281AD1604638600868264E304067
:102F5000802636033043086001990978002909D199
:102F60001660224A2A60224A2260E02219689143B0
:102F7000A03A1BE08021C9021160F2E766463E607C
:102F80000F68194E3E408027FF023E430E600199B4
:102F9000097800290DD1176001280ED1154A2A6041
:102FA000154A2260E02219689143C03A0A431A6028
:102FB000F7BD802189021160EEE7E0210F4A02434C
:102FC0002A600F4A22601A688A43F0E74B0AFF1F03
:102FD000E0000340D800034090000340000003409D
:102FE0005000034040000340FFFFE3FF0280063D26
:102FF000804508220180063D8066082200800698F0
:1030000080550822F8B51E4B80261A68002014004F
:103010003440324232D11A681A4F32431A600122C8
:103020003B68063093433B6000F07AFE0122164D68
:103030002B681E432E603B680A2613433B608027A3
:10304000BF00124B1B683B4211D1013EF6B2FF2E6E
:1030500009D17E220E4B1C682B68E40B144093436D
:1030600023432B6005E0082000F05AFEE9E7002E1C
:10307000EFD180222B68600893432B60F8BDC046D7
:10308000C4F000405CF0004018F0004068F00040E0
:1030900060F0004010B500F0EBFD01215820034A1C
:1030A00000F09EFFFFF7AEFF10BDC046600AFF1F95
:1030B00010B578220021034800F0CAFD00F0A0FFFF
:1030C000002010BDA467FF1F70B5040000F088FE4B
:1030D00000230C200B4A010059438D18515C002934
:1030E0000DD0A14208D1012300246B7000F068FDCF
:1030F00000F0EEFD200070BD01330A2BEBD112244D
:10310000F6E7C046A467FF1F70B5040000F068FE34
:10311000002319001D000D4A1078002806D0A04297
:103120000CD1557001310C320A29F5D1002B0AD18E
:1031300000F066FF00F0CCFD002070BD5078461E08
:10314000B0411B18EEE700F03BFDF3E7A467FF1F5B
:10315000F7B504000C20002384460E4D019267460B
:103160005F43E85D7E19A04212D000280BD10A4BC4
:103170009C4662461B7808331370019B70707C5527
:103180007160B360FEBD01330A2BE8D10320F9E77B
:103190000720F7E7A467FF1FA067FF1F8020F8B58F
:1031A000484BC0051B68C1248360474BFF251A6844
:1031B000012313434361454BA4001A68444B40214B
:1031C0001A60444B1A68444B1A60444B1A59AA437C
:1031D0001A51C52292009E58AE4331438026995021
:1031E0009F583F49F6010F403E439E509E5880270E
:1031F0003602360A3043985080201A5900020A409D
:1032000002431A5104341A59364E3F043240802684
:103210003A431A511A5936061202120A32431A5107
:1032200008341A5980260A4002431A51C3229200D8
:103230009F58B446AF4337439F509F58294E0F4085
:1032400007439F509F5837408026360437438026D7
:103250009F509F5836063F023F0A37439F50C02277
:103260001F59AF433A431A511A591202120A164310
:10327000C6221E5192009C58AC4365462C439C507C
:103280009C5800250C4020439850C72080001A58B5
:10329000154C1140C02212020A431A50134B1B78DE
:1032A000DB08AB4201DC0020F8BD2378002B06D000
:1032B000A368002B00D0984701350C34EEE71220AC
:1032C000F2E7C046B043FF1FAC43FF1FB0F0004021
:1032D0009C67FF1FB4F000409867FF1F00E100E00B
:1032E000FF00FFFFFFFF00FFA467FF1FA067FF1F96
:1032F000030010B51F2809D8072200201340072417
:1033000004490A78A24313430B7010BD0023062022
:10331000F5E7C046A067FF1F034A04491368002071
:103320000B4013607047C0461CF00040FFFFC1FF18
:10333000054B06491B780A6805485B0702401B0BD2
:10334000134300200B607047A067FF1F1CF0004074
:10335000FFFFC1FF70B50C25FFF7EAFF0A4B1C7891
:103360000A4BE4086543ED18002C01D1200070BD24
:103370002B78002B06D06B68002B00D09847013CBF
:103380000C3DF1E71220F2E7A067FF1F9867FF1FCF
:103390001FB5002102220B0001910091052000F0D1
:1033A00017FC02230B490A681A42FCD1202303931D
:1033B000039B5A1E0392002BFAD1074A1368002B75
:1033C000FCDA0B246C442000012100F0F9FD207888
:1033D00004B010BD90C8004000C8004013B5040000
:1033E0000A4B0193019B002B01D1112016BDFFF761
:1033F000CFFF23000340044205D0052000F090FCDD
:10340000019B013BEDE71800F0E7C046FFFFFF0717
:1034100007B500F0E5FC80220821D205936A0191EE
:10342000002B01D10739916202210C4A11600199E8
:10343000481E01900029FAD1033111600531019134
:103440000199481E01900029FAD11160002B02D188
:103450008022D205936200F03BFC07BD00C0004013
:10346000F0B52D4C89B02378002B4FD1FEF7A8FA88
:1034700002232A4F03903A681A42FCD12023069374
:10348000069B5A1E0692002BFAD1254E3368002B5C
:10349000FCDA0120FFF7A2FF011E02D0112009B0C3
:1034A000F0BD030003220190009005AD9F2000F0C5
:1034B0008FFB0321280000F083FD02233A681A42A3
:1034C000FCD120230793079B5A1E0792002BFAD1A9
:1034D0003368002BFCDA0120FFF780FF0028DDD1E4
:1034E0000398FEF781FAAA786B7811041B020B434C
:1034F00029780B4363601300113B0A49052B07D859
:1035000001239340A3600B60012323700020C6E7D2
:1035100080231B03F6E7C0469843FF1F90C8004076
:1035200000C800409808FF1F1E4B30B55A68187835
:103530001D4B85B0D31859424B4101210093002304
:1035400000F016FC194B1A4A02259A6300221A65EC
:1035500010325A658022C4219D65164B1648D2024E
:10356000DA6789004258154B80241A4080231B04D7
:1035700013434350642341200393E40500F006FA0B
:10358000402000F003FA6562039D6B1E0393002D3B
:10359000FAD103236362FFF73BFFA562FFF760FFE9
:1035A00005B030BDA443FF1F95FFFEF700C80040E3
:1035B000050001FF04E100E000E100E0FFFF00FF83
:1035C000F0B585B00700FEF7FBF9022305002D4C8E
:1035D00022681A42FCD120230093009B5A1E0092BD
:1035E000002BFAD1284E3368002BFCDA0120FFF7BC
:1035F000F5FE002803D01124200005B0F0BD234BB8
:103600002360022322681A42FCD120230193019BEC
:103610005A1E0192002BFAD13368002BFCDA0120EC
:10362000FFF7DCFE0028E6D1194B1F600223226859
:103630001A42FCD120230293029B5A1E0292002BB5
:10364000FAD13368002BFCDA0120FFF7C7FE00280F
:10365000D1D1104B2360022322681A42FCD12023CF
:103660000393039B5A1E0392002BFAD13368002B5D
:10367000FCDA0120FFF7B2FE041EBCD12800FEF7E1
:10368000B3F9B9E790C8004000C800400100000647
:10369000A8C800400180000110B50020FFF790FF8E
:1036A00010BD000010B5064B18705960FFF73CFFC5
:1036B00000211320034AFFF74BFD002010BDC04638
:1036C000A443FF1F2935FF1FF0B5040085B0039206
:1036D0000291FEF775F9882263035B0B52051A43CA
:1036E0008023DB059D6A8023274F0092BA6800265D
:1036F00001901B039A420CD9F82326001B041E409C
:103700001C4206D08022214B52025E6219680A4395
:103710001A60002D0BD100F063FB02221C4B1A60D3
:103720008023DB055A62013A9A6200F0D1FA002345
:10373000039A934220D1002D0AD100F051FB144B83
:1037400003221D608023DB055A629D6200F0C0FAEF
:103750008023BA681B039A4208D9002E06D00022A3
:103760000A4B0C495A621A680A401A600198FEF71F
:103770003BF9002005B0F0BD009A0299D2181278EA
:10378000CA540133D4E7C0469843FF1F00C8004025
:1037900000C00040FFFFFEFFF0B587B0029103922A
:1037A0000400FEF70DF9019000F01AFB80230225BA
:1037B0000122234EDB0535605D629A6200F088FAD3
:1037C000204F3B682B42FCD120230493049B5A1EBC
:1037D0000492002BFAD11C4D2B68002BFCDA01203F
:1037E000FFF7FCFD002802D0112007B0F0BD20003B
:1037F000039A029900F0CCFA022304003A681A42B4
:10380000FCD120230593059B5A1E0592002BFAD16B
:103810002B68002BFCDA0120FFF7E0FD051EE3D149
:1038200000F0DEFA80230322DB0535605A629D62D8
:1038300000F04EFA0198FEF7D7F8E0B2D5E7C0469F
:1038400000C0004090C8004000C80040F0B580248F
:1038500089B00600FEF7B4F8E405A36A02250393D5
:10386000029000F0BDFA0123304F3D606562A36213
:1038700000F02EFA2E4C23682B42FCD12023059316
:10388000059B5A1E0592002BFAD12A4D2B68002B5E
:10389000FCDA0120FFF7A2FD002803D0112420004C
:1038A00009B0F0BD244B2360022322681A42FCD1E8
:1038B00020230693069B5A1E0692002BFAD12B68F2
:1038C000002BFCDA0120FFF789FD021EE6D11B4B1D
:1038D00003211E60030001900090202000F078F981
:1038E000022322681A42FCD120230793079B5A1E09
:1038F0000792002BFAD12B68002BFCDA0320FFF78C
:103900006DFD041ECAD100F06BFA80230322DB0593
:103910003C605A629C6200F0DBF9039B002B01D1F2
:10392000FFF776FD0298FEF75FF8B8E700C00040A9
:1039300090C8004000C800400100000694C8004044
:1039400007B5000201910422000A01A9FFF724FF34
:103950000EBD000073B5050005240B4AA3005B42B1
:103960009B1819686B46DE1D3000FFF7A7FA022886
:1039700004D133782B55013CEFD276BD052CFCD019
:103980000128FAD10230F8E7140900111F2807D8DE
:10399000012380228340D20591680B4393607047D6
:1039A0003F2808D80123802220388340D20551695E
:1039B0000B435361F3E75F28F1D80123802240389D
:1039C0008340D205116A0B431362E8E71F2807D82A
:1039D000012280218240C9058B6893438B60704728
:1039E0003F2808D80122802120388240C9054B6930
:1039F00093434B61F3E75F28F1D8012280214038DF
:103A00008240C9050B6A93430B62E8E71F2810D870
:103A100080230200DB05153A1968012A06D8202206
:103A20009143196019680A431A6070470122824065
:103A3000F6E73F2811D880230200DB05353AD96824
:103A4000032A06D810229143D960D9680A43DA6064
:103A5000EBE7012220388240F5E75F28E5D84223D2
:103A60008022181A413B8340D205516A9943516222
:103A7000516A0B435362D8E710B50400012813D1F3
:103A8000A022184992050B685B015B0913430B6088
:103A9000154B164A19681140154A0A431A6040220C
:103AA00019680A431A6010BD0028FCD101000A20E1
:103AB00000F0E6F821000B2000F0E2F8C0220A4BEB
:103AC000920019680A4340211A601A688A431A60F2
:103AD000B022044912060B685B015B0913430B60BB
:103AE000E1E7C04614F000401CF000407F00FEFFFC
:103AF00080FD010072B6074A136801331360042287
:103B0000054B1A600023054A13608022D2055360DA
:103B1000FEE7C0467808FF1FC0F00040C4F0004038
:103B200005490B68002B05D1044A0A6004490A6064
:103B3000044A13607047C046140AFF1F841E000029
:103B4000380AFF1FC4F000400023034A1360034AF1
:103B50001360034A1360704754F0004040F1004086
:103B600044F1004002B47146490849000956490031
:103B70008E4402BC7047C04602B4714649084900F1
:103B8000095C49008E4402BC7047C04603B47146CC
:103B9000490840004900095A49008E4403BC704757
:103BA00001B40248844601BC604700BFED6B0100D0
:103BB00001B40248844601BC604700BFE927000009
:103BC00001B40248844601BC604700BF21A900003F
:103BD00001B40248844601BC604700BF496D010042
:103BE00001B40248844601BC604700BF156B010068
:103BF00001B40248844601BC604700BF016C01006B
:103C000001B40248844601BC604700BF2D6C01002E
:103C100001B40248844601BC604700BFF935010089
:103C200001B40248844601BC604700BF7997000098
:103C300001B40248844601BC604700BFF90D010091
:103C400001B40248844601BC604700BF2144000023
:103C500001B40248844601BC604700BFB70E0000B3
:103C600001B40248844601BC604700BFC95C010042
:103C700001B40248844601BC604700BFED68010002
:103C800001B40248844601BC604700BFEDA30011A7
:103C900001B40248844601BC604700BFCD4C01001E
:103CA00001B40248844601BC604700BFBD0B01005F
:103CB00001B40248844601BC604700BFE917010017
:103CC00001B40248844601BC604700BF8D11010069
:103CD00001B40248844601BC604700BF9DA90000B2
:103CE00001B40248844601BC604700BF613701004F
:103CF00001B40248844601BC604700BFD9B000004F
:103D000001B40248844601BC604700BF116E000048
:103D100001B40248844601BC604700BF89440000EA
:103D200001B40248844601BC604700BF018900001D
:103D300001B40248844601BC604700BF85520100BF
:103D400001B40248844601BC604700BFC1A5000021
:103D500001B40248844601BC604700BF8B52010099
:103D600001B40248844601BC604700BFE9D40000AA
:103D700001B40248844601BC604700BFC56D010024
:103D800001B40248844601BC604700BF75F80000DA
:103D900001B40248844601BC604700BF957301002E
:103DA00001B40248844601BC604700BF851201008F
:103DB00001B40248844601BC604700BF791201008B
:103DC00001B40248844601BC604700BFB352010001
:103DD00001B40248844601BC604700BF5976010027
:103DE00001B40248844601BC604700BF75A90000C9
:103DF00001B40248844601BC604700BFA9D8000056
:103E000001B40248844601BC604700BF85C1000080
:103E100001B40248844601BC604700BFBD5C01009C
:103E200001B40248844601BC604700BF71B0000085
:103E300001B40248844601BC604700BF53B900008A
:103E400001B40248844601BC604700BFE51201008E
:103E500001B40248844601BC604700BFA1AF000026
:103E600001B40248844601BC604700BFD1AE0000E7
:103E700001B40248844601BC604700BFF9ED000070
:103E800001B40248844601BC604700BFC9A90000D4
:103E900001B40248844601BC604700BF6D0B0100BD
:103EA00001B40248844601BC604700BFE9F6000047
:103EB00001B40248844601BC604700BF01D700003E
:103EC00001B40248844601BC604700BFDD3F0000EA
:103ED00001B40248844601BC604700BF0D52010096
:103EE00001B40248844601BC604700BFDD0A0100FE
:103EF00001B40248844601BC604700BF71B700119D
:103F000001B40248844601BC604700BF8D820000B6
:103F100001B40248844601BC604700BF9D6A0000AE
:103F200001B40248844601BC604700BF013401006F
:103F300001B40248844601BC604700BFE90B0100A0
:103F400001B40248844601BC604700BF19FA000072
:103F500001B40248844601BC604700BF69110100FA
:103F600001B40248844601BC604700BF6DF6000002
:103F700001B40248844601BC604700BFC16601002D
:103F800001B40248844601BC604700BF090E00002E
:103F900001B40248844601BC604700BF51B800002C
:103FA00001B40248844601BC604700BFF5350100FA
:103FB00001B40248844601BC604700BFDD0C01002B
:103FC00001B40248844601BC604700BF3D71010056
:103FD00001B40248844601BC604700BFC1F700003D
:103FE00001B40248844601BC604700BF016701007C
:103FF00001B40248844601BC604700BFE94C01009F
:1040000001B40248844601BC604700BFADAE000069
:1040100001B40248844601BC604700BF053401007A
:1040200001B40248844601BC604700BFC1150100CD
:1040300001B40248844601BC604700BF89140100F6
:1040400001B40248844601BC604700BFEDA50000F2
:1040500001B40248844601BC604700BFCD0C01009A
:1040600001B40248844601BC604700BF89370100A3
:1040700001B40248844601BC604700BFD54401003A
:1040800001B40248844601BC604700BF0934010006
:1040900001B40248844601BC604700BF4DF90000EE
:1040A00001B40248844601BC604700BF090E00000D
:1040B0000200000066C000110100000038BE0011BF
:1040C0000200000062C0001101000000F040FF1F6C
:1040D0000200000040BE0011010000002C62FF1F22
:1040E0000200000060C0001103000000A061FF1F7B
:1040F000120000000200000066C000110100000074
:1041000080BE00110200000062C00011010000002A
:104110007DBE0011020000008ABE001103000000F5
:10412000DB61FF1F0200000060C0001103000000FF
:10413000F061FF1F0200000062C0001101000000DA
:104140007CBE00110200000088BE001103000000C8
:10415000B161FF1F0200000060C0001103000000F9
:10416000D261FF1F0200000066C0001101000000C4
:10417000C4BE00110200000062C000110100000076
:104180003942FF1F02000000D6BE001101000000EE
:10419000BBBE00110200000062C00011010000005F
:1041A0003842FF1F02000000D4BE001101000000D1
:1041B000F861FF1F0200000062C000110100000052
:1041C0003742FF1F02000000D2BE001101000000B4
:1041D000ABBE00110200000062C00011010000002F
:1041E0003642FF1F02000000D0BE00110100000097
:1041F000A6BE00110200000062C000110100000014
:104200003542FF1F02000000CEBE00110100000079
:10421000A1BE00110200000062C0001101000000F8
:104220003442FF1F02000000CCBE0011010000005C
:104230009CBE001102020202020200000000000007
:1042400014130000CD4C0011934C001134BF001129
:1042500090011D0018001800FFFF0701020304056C
:10426000060201060000000000000000000000003F
:10427000000000000000000000000000000000003E
:10428000030000000200000066C0001101000000F1
:1042900054BF00110200000062C0001101000000C4
:1042A000F442FF1F020000005EBF00110100000089
:1042B0002662FF1F0200000060C000110300000022
:1042C0009064FF1F0200000062C0001101000000A6
:1042D000F442FF1F020000005CBF0011010000005B
:1042E0002862FF1F0200000060C0001103000000F0
:1042F0008864FF1F12006C6C0000000000000000CA
:10430000000000000807000000010000000001118B
:10431000FFFF000050485936000000000000000078
:104320000B000500F0000000B40000280028002861
:104330003075A000A000A000A00000080008E00167
:10434000F0001000100010001000100010005000CD
:104350005000500010001000D007000000000000C6
:104360000F0001000500307507001000010081FFFB
:1043700000000000FF000000D5750011DD73001182
:104380006D710011FFFF0100FF000000F19F00119F
:104390006D9D0011859C00110000000000000000D0
:1043A00000000800040000003B0001085902E00181
:1043B00088212800FF0000000200000066C00011F4
:1043C000010000002CC100110200000062C00011B9
:1043D000010000003544FF1F020000005EC0001114
:1043E000010000005C68FF1F0200000062C00011B5
:1043F000010000003444FF1F020000005CC00011F7
:10440000010000003244FF1F0200000062C00011E2
:10441000010000003044FF1F020000005AC00011DC
:10442000010000002844FF1F180018001D00900123
:1044300002000003020200000200000066C000113A
:104440000100000040C100110200000062C0001124
:10445000010000007844FF1F0200000058C0001156
:1044600000000000000000000200000060C0001119
:0A447000030000007C68FF1F20FF1E
:040000051FFF184180
:00000001FF
